:030000000252FAAF
:0C52FA0078FFE4F6D8FD75817F02534177
:1024810020000A3C2E2E2E3E004950436F6E6E6591
:1024910063745245510A004950436F6E6E6563740F
:1024A100000A49504E6F41434B210A003E432C56CE
:1024B1002C52432CC0E4E0EFF2E5F020D1E8EDEA44
:1024C100EEEC49500A003E432C4D41432C2530325D
:1024D10062583A25303262583A25303262583A25EC
:1024E100303262583A25303262583A2530326258D9
:1024F1002C4D414320E0E4F0E5F10A003E432C5627
:1025010045522C20332E3220EEF2202573202573E4
:102511002CC2E5F0F1E8FF20495020ECEEE4F3EBAA
:10252100FF0A0041707220323420323031330031E1
:10253100353A33383A3134003E432C4C442C505216
:102541004F473A202020202020202020202020201A
:10255100202020202020202020202020202020207A
:10256100202020202020202020202020202020206A
:10257100202020202020202020202020202020205A
:1025810020202020202020202CC4E0F2E020EFF0A9
:10259100EEF8E8E2EAE828F4E0E9EB290A003E2A4D
:1025A1002C312CCEF1EDEEE2EDFBE520EFE0F0E099
:1025B100ECE5F2F0FB20F1E5F2E5E2EEE3EE20E8F6
:1025C100EDF2E5F0F4E5E9F1E00A003E412C41309D
:1025D100312C2562752E2562752E2562752E256298
:1025E100752C495020E0E4F0E5F120E0E4E0EFF261
:1025F100E5F0E00A003E412C4130322C2562752E77
:102601002562752E2562752E2562752C495020E0B4
:10261100E4F0E5F120EEF1ED2E20F1E5F0E2E5F058
:10262100E00A003E412C4130332C2562752E256293
:10263100752E2562752E2562752C495020E0E4F037
:10264100E5F120F0E5E72E20F1E5F0E2E5F0E00A22
:10265100003E412C4130342C2562752E2562752EA9
:102661002562752E2562752CCCE0F1EAE020F1E5BA
:10267100F2E80A003E412C4130352C2562752E25A9
:1026810062752E2562752E2562752CD8EBFEE70A40
:10269100003E2A2C312CC4EEEF2E20EFE0F0E0ECCE
:1026A100E5F2F0FB20F1E5F2E5E2EEE3EE20E8ED04
:1026B100F2E5F0F4E5E9F1E00A003E422C53303254
:1026C1002C2562752CCEE1ECE5ED20F120F1E5F051
:1026D100E2E5F0EEEC20E1E5E720EAE2E8F2E0ED08
:1026E100F6E8E90A003E422C5330332C2562752C62
:1026F100CFE5F0E5E7E0EFF3F1EA20EFF0E820EFD6
:10270100EEF2E5F0E520F1E2FFE7E820F120F1E566
:10271100F0E2E5F0EEEC0A003E422C5330382C2575
:1027210062752CCCE5E4EBE5EDEDFBE920495020A9
:10273100EAE0EDE0EB28E7E0E4E5F0E6EAE020E4BA
:10274100EE203520F1E5EA290A003E422C533035CE
:102751002C2562752CCAE0EDE0EB20F8E8F0EEEAFA
:10276100EEE2E5F8E0F2E5EBFCEDEEE3EE20EEE182
:10277100ECE5EDE00A003E532C5330362C25303287
:102781006258253032625825303262582530326223
:1027910058253032625825303262582C4D41432041
:1027A100E0E4F0E5F120F8E8F0EEEAEEE2E5F8E049
:1027B100F2E5EBFCEDEEE3EE20EEE1ECE5EDE00A17
:1027C100003E454E440A000A44756D705820202091
:1027D100202030302030312030322030332030344E
:1027E1002030352030362030372030382030392025
:1027F10030412030422030432030442030452030C9
:1028010046000A3A003A20000A000A44756D7044F5
:102811002020202020303020303120303220303331
:1028210020303420303520303620303720303820E9
:102831003039203041203042203043203044203094
:102841004520304600457272206B65790052642044
:10285100656570726F6D0A005264204D454D0A0026
:10286100526420436F64650A00577269746520439E
:102871006F64650A0044656275674950204F4E0ACE
:102881000044656275674950204F46460A00446519
:1028910062756755736572204F6E0A0044656275F3
:1028A1006755736572204F46460A00446562756735
:1028B1004D7367204F6E0A0044656275674D7367FB
:1028C100204F46460A00436F6E666967206C6F634E
:1028D1006B210A00577220656570726F6D0A0020C6
:1028E1005361766520656570726F6D210A004572CE
:1028F10072204D414321004C6F61643E3E002A002D
:10290100CEF8E8E1EAE00A00202D2025752825759A
:10291100290A003C4130313D003C4130323D003C10
:102921004130333D003C4130343D003C4130353D88
:10293100003C21003C5330323D003C5330333D00DC
:102941003C5330353D003C5330383D003C5330362C
:022951003D0047
:065CFA000113000111007E
:105EA100C28E438910E4F58B758DB8D2ABD28E22A8
:03001B000251DBB4
:1051DB00C0E0C083C082C0D0C28E758B00758DB805
:1051EB0020280675A61E75A6E10511D224E51360CD
:1051FB000205130516E516540F7051E512D39401F1
:10520B0040021512D230E516543F7012D222907F15
:10521B0069E0600A04F0E0D394B44002D228907F96
:10522B0062E0600204F09079DFE0600214F0907F9E
:10523B006AE0D394014003E014F03027020514E533
:10524B0015D394644004D22880020515E510D3943D
:10525B000140021510D28ED0D0D082D083D0E03254
:101EAA00C22D7D027C007F07125DF98F28E5286428
:101EBA006060097D017F60125D71D22DE4FDFC7FB7
:101ECA000B125DF98F28E52830E6097D04E4FF123C
:101EDA005D95D22D7D017C007F07125DF98F28E583
:101EEA00287008FD7FFF125D71D22D302D0312601C
:101EFA0000C288C2A8C2AA75890012513F907C25E7
:101F0A007403F0A374CCF0E4907C24F0907F67F023
:101F1A00A3F0124D8F124FDCC2281258F0D22DC2F4
:101F2A002FC22E907E527408F0907B907424F0E4B5
:101F3A00A3F0907C1AE0907B92F0907C1BE0907B5F
:101F4A0093F0907C1CE0907B94F0907C1DE0907B59
:101F5A0095F0907C1EE0907B96F0907C1FE0907B41
:101F6A0097F0751201E4907E53F0C229C22AC22B5F
:101F7A00C22C202D18AF28FE7D03124BD3E4FF128A
:101F8A00508F7E247F81E4FBFDFC1248E0907F693C
:101F9A00E060037401F0E49079DFF0F514907E516B
:101FAA00F0F515125EA175A70775A61E75A6E1D2F2
:101FBA00AFC225E4F5159079DFE0700312179D9002
:101FCA007F6AE06401701D9080007410F09080A810
:101FDA0074FFF0A3F0A3F0A3F0E4907F6AF0D22D8F
:101FEA00C22EC22F908008E0F52830E405D2297469
:101FFA0010F0E52830E508D22B9080087420F0E52F
:10200A002830E608D22A9080087440F0E514C39478
:10201A00034019908002E4F0908001F0908000F073
:10202A00E51494064006E4F5141258F09080A0E0F6
:10203A00700312569C9080B8E0700312562290806A
:10204A00D0E07003125894908000E0701330291089
:10205A001249E7907C0DEFF0D3940040031200364A
:10206A00908002E07006908000E06005D227021F8F
:10207A00BDC227E4F5149079DFE06003021FBD209A
:10208A002D12907E54E0600C7E247F83124AEBE48A
:10209A00907E54F0302B12124288907C0DEFF0D3D0
:1020AA0094004005E0FF12107D202A030222361216
:1020BA003F83907C0DEFF07003021FBD907C51E0CE
:1020CA0054BF247F700302219114700302216924F2
:1020DA000260030221D8202D077E247F8A124AEB50
:1020EA00907C29E0FF7006907C2DE06061907F5E15
:1020FA00E0FEB50722A3E0FF907C2AE0B50718901E
:10210A007F60E0FF907C2BE0B5070C907F61E0FFD9
:10211A00907C2CE06F6037907C2DE06E6003022289
:10212A0036907F5FE0FF907C2EE06F6003022236DC
:10213A00907F60E0FF907C2FE06F60030222369070
:10214A007F61E0FF907C30E06F6003022236C22597
:10215A00907E537401F0125F1475120102223690B8
:10216A007F69E060037401F0907F56E0FF907C5332
:10217A00E06F6003022236907F56E004F0E4F51225
:10218A00907E51F0022236302503022236907C20BE
:10219A00E07003021FBD907B8FE06008907C317471
:1021AA001EF08006907C317403F0125F13D225E48E
:1021BA00F512907E51F0907F6204F0E4907F55F022
:1021CA00A3F0202D677E247F98124AEB805E907FD1
:1021DA0069E060037401F0302552907C51E020E7F9
:1021EA004B907C53E0FF907F55E0FE6F600D907F2F
:1021FA005DE07007EE146F70338013907F55E00432
:10220A00F0907C0DE0FFD3940440031200329078E2
:10221A00DB7482F0A37401F0907C53E09078DDF0D7
:10222A007E787FDB7D0312540D021FBD2025030239
:10223A002359E512706E125C42EF60237E7D7F5156
:10224A00907D52E02404FD12540D907F5DE07009E8
:10225A00907C31E0F512021FBDE4F512021FBD9019
:10226A007F62E0D3943C403C907F5DE07036907B87
:10227A008FE07030907F6204F0124F27E4907D5116
:10228A00F0A37412F0907F56E0907D53F0A374FD92
:10229A00F09079E063A201907D5563A2017F12124A
:1022AA003CD18098125F018F28E528B401159078F7
:1022BA00DB7483F0E4A3F07E787FDB7D0212540D99
:1022CA00021FBDE528D39401401C9078DB7483F08B
:1022DA00A37401F0E52824FEA3F07E787FDB7D035A
:1022EA0012540D021FBDE51264016003021FBD9066
:1022FA007E51E004F0202D077E247FA2124AEB9043
:10230A007E51E0FFD39401400B907C31E0941E5043
:10231A0003E004F0EFC39405400DC225E4907E5318
:10232A00F0125F14021FBD7C7F7D5E907C25E0FA6F
:10233A00A3E0FB7F0212559E7E7D7F51907D52E085
:10234A002404FD12540D907C31E0F512021FBDE504
:10235A001264016003021FBD907E53E0146065148D
:10236A0070030224621470030224702403600302BF
:10237A001FBDE4F514907F5DE06020907C29E0FCAD
:10238A00A3E0FDA3E0FEA3E0FF907F5E122C59902C
:10239A007C257403F0A374CCF0802930B40E907EAF
:1023AA00537402F0751203D2B5021FBD90800274F5
:1023BA0010F0907E517401F0751212907F5E74FFD6
:1023CA00F0021FBD907F5EE0605D907D517480F0E9
:1023DA00907D537401F0E4A3F0A304F0A3743FF0DA
:1023EA00A3747BF0E4F52874582528F582E4347D3B
:1023FA00F583747DF074592528F582E4347DF583DC
:10240A00E4F0E5282407907D52F07C7F7D5E907C85
:10241A0025E0FAA3E0FB7F0212559E7E7D7F51E5FF
:10242A00282409FD12540D907F5DE06020E4907E1F
:10243A0053F0125F13D225E4F512907E51F0907F8B
:10244A006204F0E4907F55F0A3F0021FBDE4907E91
:10245A0053F0751212021FBD907E537402F075126A
:10246A0003C2B5021FBDE4907E53F01258F07512F4
:06247A0012021FBD80FEEE
:012480002239
:10003600907C52E0B444047F0180027F00907C51A2
:10004600E0B447047E0180027E00EE5F604A907C49
:100056001AE0907C53F0907C1BE0907C54F0907CEE
:100066001CE0907C55F0907C1DE0907C56F0907CD6
:100076001EE0907C57F0907C1FE0907C58F0907CBE
:10008600527452F0907B8963A2019080A863A2010A
:100096007F06123CD1020904907C0DE0C3940850FF
:1000A6000302090D907C1AE0FF907C53E06F600319
:1000B60002090D907C1BE0FF907C54E06F60030208
:1000C600090D907C1CE0FF907C55E06F60030209EF
:1000D6000D907C1DE0FF907C56E06F600302090DD9
:1000E600907C1EE0FF907C57E06F600302090D9044
:1000F6007C1FE0FF907C58E06F600302090D907C46
:1001060052E06444701A9080A8E0B4FF13907B8993
:1001160063A2019080A863A2017F06123CD18010E1
:10012600907B8DE09080ACF0907B8EE09080ADF07F
:10013600907F69E060037401F0907F6A7464F090C8
:100146007C527452F0907C51E0646D60030202AB05
:100156007BFF7A2479AD12316D7BFF7A2479C790C3
:100166007C1AE0F535A3E0F536A3E0F537A3E0F514
:1001760038A3E0F539A3E0F53A12316D7535FF7510
:1001860036257537247538FF753925753A307BFF66
:100196007A2479FD12316D7BFF7A25793912316D1A
:1001A6007BFF7A25799F12316D7BFF7A2579CC907A
:1001B6007C20E0F535A3E0F536A3E0F537A3E0F5BE
:1001C6003812316D7BFF7A2579F6907C29E0F5357A
:1001D600A3E0F536A3E0F537A3E0F53812316D7BE1
:1001E600FF7A267924907C2DE0F535A3E0F536A339
:1001F600E0F537A3E0F53812316D7BFF7A267952A8
:10020600907C16E0F535A3E0F536A3E0F537A3E0DC
:10021600F53812316D7BFF7A267975907C12E0F500
:1002260035A3E0F536A3E0F537A3E0F53812316DD6
:100236007BFF7A26799212316D7BFF7A2679BB9005
:100246007F5DE0F53512316D7BFF7A2679E6907F8A
:1002560069E0F53512316D7BFF7A277919907B8F2E
:10026600E0F53512316D7BFF7A27794BA223E43313
:10027600F53512316D7BFF7A277977907F57E0F558
:1002860035A3E0F536A3E0F537A3E0F538A3E0F5AE
:1002960039A3E0F53A12316D1239E87BFF7A2779F6
:1002A600C212316D22907C51E0644C70737E277FC0
:1002B600C8FBFDFC1248E0907C59E0F529A3E0F567
:1002C6002AE4F52CE529907C5BF0A3E52AF07E284C
:1002D6007F037C7C7D5B7B021248E0E4F52B852A5C
:1002E60082852983E0FF745B252BF582E4347CF557
:1002F60083EFF0052AE52A70020529052BE52BB4C4
:1003060010DC7E287F067C7C7D5B7B101248E00536
:100316002CE52CC3941040AC7E287F09124AEB22B0
:10032600907C51E0646C7060F52D7E287F0BFBFDA0
:10033600FC1248E0E4F52CE4907C5BF0A3E52DF09C
:100346007E287F037C7C7D5B7B021248E0E4F52BF4
:10035600A82DE6FF745B252BF582E4347CF583EF4C
:10036600F0052D052BE52BB410E67E287F067C7C58
:100376007D5B7B101248E0052CE52CC3940840B742
:100386007E287F09124AEB22907C51E0644B706113
:10039600F52B7443252BF582E4347CF583E060323B
:1003A6007443252BF582E4347CF583E0F4602374F2
:1003B60043252BF582E4347CF583E0FF7459252B25
:1003C600F582E4347CF583E0B50710052BE52BB404
:1003D60008C09079DF7432F0020904907C517421D0
:1003E600F0302D030209047E287F46124AEB0209EB
:1003F60004907C51E0B4521A202D077E287F4E12BD
:100406004AEB907C517472F07E7C7F517D081253CA
:100416008622907C51E064497045202D077E287F16
:1004260059124AEB907C59E0F529A3E0F52AE4F548
:100436002B852A82852983E0FF745B252BF582E4D0
:10044600347CF583EFF0052AE52A70020529052B91
:10045600E52BB480DC7E7C7F517D8A125386229008
:100466007C51E064437046202D077E287F61124A46
:10047600EB907C59E0F529A3E0F52AE4F52B852AD3
:1004860082852983E493FF745B252BF582E4347C13
:10049600F583EFF0052AE52A70020529052BE52BE1
:1004A600B480DB7E7C7F517D8A12538622907C51FC
:1004B600E0645A7053202D077E287F6A124AEB901B
:1004C6007C59E0F529A3E0F52A7C7C7D5B7B80AF37
:1004D6002AAE29125C0EE4F52B852A82852983E44F
:1004E60093FF745B252BF582E4347CF583EFF005EE
:1004F6002AE52A70020529052BE52BB480DB7E7CD4
:100506007F517D8A12538622907C51E064446003B9
:1005160002059F907C59E0FF64447003020904EFD2
:10052600B4310CC22D7E287F76124AEB0209049064
:100536007C59E0B4300CD22D7E287F82124AEB0221
:100546000904907C59E0B4320CD22E7E287F8F129B
:100556004AEB020904907C59E0B4330CC22E7E2883
:100566007F9D124AEB020904907C59E0B4340CD208
:100576002F7E287FAC124AEB020904907C59E0B426
:10058600350CC22F7E287FB9124AEB020904907CF3
:1005960059E0FF125E7B0209049079DFE0701320B8
:1005A6002D077E287FC7124AEB907C517421F002FA
:1005B60009049079DF7432F0907C51E0FFB4510465
:1005C600C2AF80FEEF64577045202D077E287FD589
:1005D600124AEB907C5AE0907C0DF0E4F52B907C6F
:1005E6000DE0FFE52BC39F4003020904745B252B36
:1005F600F582E4347CF583E0FF907C59E0252B24DA
:1006060088F582E4347AF583EFF0052B80D0907C70
:1006160051E0645360030206C1202D077E287FE067
:10062600124AEB907C1AE0FF907A91E06F703C9052
:100636007C1BE0FF907A92E06F7030907C1CE0FFAC
:10064600907A93E0B50724907C1DE0FF907A94E0C1
:10065600B50718907C1EE0FF907A95E0B5070C90E0
:100666007C1FE0FF907A96E06F6016907C517421B3
:10067600F0302D030209047E287FEF124AEB0209AF
:1006860004E4F52BE4F5157488252BF582E4347A19
:10069600F583E0FDAF2B125CD0052BE52BC394FE52
:1006A60040E2C2AFE4907FF0F0A3F0907FFD74AA21
:1006B600F0A374FFF0A37455F080FE907C51E064C3
:1006C6004F705A907C59E0F529A3E0F52AE52A45B2
:1006D60029700A202D077E287FF8124AEB202D0765
:1006E6007E287FFF124AEBE4F52B745B252BF582FF
:1006F600E4347CF583E0852A82852983F0052AE5A2
:100706002A70020529052BE52BB480DE907F68E070
:100716002480F0907F67E03400F0020904907C5159
:10072600E064457074907C59E0FEA3E0FF907FF092
:10073600EEF0A3EFF0D39400EE94044038907FF0EF
:10074600E0FEA3E0FF907F67E0FCA3E0FD9FEC9E48
:100756004023E42FFFEE3401FED3ED9FEC9E5015AF
:10076600C2AF907FFD74AAF0A374FFF0A37455F096
:10077600E4F5A780FE7E297F01124AEB7BFF7A29EA
:100786007909907FF0E0F535A3E0F536907F67E0D4
:10079600F537A3E0F53812316D907C51E064656061
:1007A6000302090D907C59E0FFA3E0907FF0CFF0A3
:1007B600A3EFF0E4F529F52AD3907FF1E0952A908E
:1007C6007FF0E095294021E4F515252AFFE5293437
:1007D60078FE7B80AD2AAC29125C0E7480252AF542
:1007E6002AE43529F52980D07E297F14125494EF06
:1007F6004E6020120003907C20EFF0120003907CE4
:1008060021EFF0120003907C22EFF0120003907C9F
:1008160023EFF07E297F1A125494EF4E60201200C7
:1008260003907C29EFF0120003907C2AEFF012006F
:1008360003907C2BEFF0120003907C2CEFF07E29C6
:100846007F20125494EF4E6020120003907C2DEF0F
:10085600F0120003907C2EEFF0120003907C2FEF35
:10086600F0120003907C30EFF07E297F261254941C
:10087600EF4E6020120003907C16EFF012000390FA
:100886007C17EFF0120003907C18EFF01200039033
:100896007C19EFF07E297F2C125494EF4E602012C3
:1008A6000003907C12EFF0120003907C13EFF0121D
:1008B6000003907C14EFF0120003907C15EFF0E437
:1008C600F52BE4F515E52B04FF7412252BF582E4D0
:1008D600347CF583E0FD125CD0052BE52BC39443F5
:1008E60040E0C2AFE4907FF0F0A3F0907FFD74AAE1
:1008F600F0A374FFF0A37455F0E4F5A780FE7E7CA8
:070906007F517D08125386AA
:01090D0022C7
:105BD600AE07EEC39430400BEED394395005EE2455
:105BE600D0FF22EEC39461400BEED394665005EECF
:105BF60024A9FF22EEC39441400BEED394465005F0
:085C0600EE24C9FF22AF0622C3
:105E3300907B88E004F07006907B87E004F0907B11
:0A5E430087E0FEA3E0FF125B572288
:10000300125E33125BD6EFC454F0FEC006125E33A9
:08001300125BD6D0E02FFF22A2
:10583700E4907F72F0125E33907F73EFF0C3943081
:105847004018E0FFD394395011907F72E024E0F5BF
:1058570082E43479F583EFF08011907F72E024E0E1
:10586700F582E43479F583E4F0800C907F72E004EC
:10587700F0E0D3940840BE753100753200753300EF
:0C588700E4F5347B017A7979E0123DDF12
:0158930022F2
:045494008E2E8F2F9A
:10549800907B87E4F0A374FFF0125E33EF606EF444
:1054A800606B852F82852E83E493B507EC753001F8
:1054B800E52F2530F582E4352EF583E493602590B9
:1054C8007B88E02530FF907B87E03400FE125B5735
:1054D800E52F2530F582E4352EF583E493B50704EE
:1054E800053080CCE52F2530F582E4352EF583E4B0
:1054F8009370A6E53024FFFFE434FFFE907B88E03C
:105508002FF0907B87E03EF07E007F0122E4FEFFD3
:015518002270
:104D8F007E297F32125494EF4E70037F01227E29C9
:104D9F007F35125494EF4E600C125E33EF24D09097
:104DAF007F5DF08005E4907F5DF07E297F3B12549C
:104DBF0094EF4E600C125E33EF24D0907F69F08039
:104DCF0005E4907F69F07E297F41125494EF4E6085
:104DDF000C125E33EF24D024FF92238002C2237E75
:104DEF00297F47125494EF4E600C125E33EF24D09C
:104DFF00907B8FF08005E4907B8FF0907C1A63A2FC
:104E0F0001907F5763A2017F06123CD130233B7E76
:104E1F00297F4D125494EF4E6030120003907F574C
:104E2F00EFF0120003907F58EFF0120003907F59BC
:104E3F00EFF0120003907F5AEFF0120003907F5BA8
:0D4E4F00EFF0120003907F5CEFF07F002277
:105A4000907E52E0C3947C40027F0A907E52E0FE3A
:105A500004F074902EF582E4347BF583EFF0BF0AF6
:105A600027907E52E0FF04F074902FF582E4347B9F
:105A7000F583E4F0907E52E0FF125519907E527447
:095A800008F0907B91E004F02293
:1058F0009080007480F0907C1263A201F583F582A1
:1059000063A2017F08123CD1907C1A63A2019080AF
:105910008863A2017F0A123CD19080927407F0A3A1
:1059200074D0F0A37406F0907C24E0FF9080B1F076
:105930009080E1EFF09080957455F0A3F090800096
:0A5940007401F090800974F0F02269
:10569C00908009E04410F09080A0E070609080A1B0
:1056AC007482F09080A874FFF0A3F0A3F0A3F07FB5
:1056BC00039080AEEFF0A374CBF09080007402F0F6
:1056CC00907FD3122C6500000000907FD3E0908077
:1056DC0040F0907FD4E0908041F0907FD5E09080B6
:1056EC0042F0907FD6E0908043F0A3E4F0A3F0A3C7
:0D56FC00F0A3F0908018F0A3F0A3F0A3F04D
:01570900227D
:10589400908009E04440F09080D17482F07F0390BE
:1058A40080DEEFF0A374CCF09080027402F0907F5D
:1058B400D7122C6500000000907FD7E0908058F04C
:1058C400907FD8E0908059F0907FD9E090805AF092
:1058D400907FDAE090805BF0A3E4F0A3F0A3F0A360
:0B58E400F0908030F0A3F0A3F0A3F0E0
:0158EF002296
:10562200908009E04420F09080B8E0706C9080B9DE
:105632007482F07F039080C6EFF07FCDA3EFF07FFE
:10564200039080C4EFF0A374CDF09080C074FFF09B
:10565200A3F0A3F0A3F09080017402F0907FDB121C
:105662002C6500000000907FDBE090804CF0907F82
:10567200DCE090804DF0907FDDE090804EF0907FF6
:10568200DEE090804FF0A3E4F0A3F0A3F0A3F0904B
:095692008024F0A3F0A3F0A3F0C2
:01569B0022EC
:10559E008C298D2AA907EAFDE975F018A424ACFF21
:1055AE00E5F034808F82F583EDF0EBFDE975F018B0
:1055BE00A4FFAEF024ACFBEE34808B82F583A3ED1A
:1055CE00F0852A828C83E0FDEF24A8FFEE3480FE66
:1055DE008F82F583EDF0852A828C83A3E08F828EF5
:1055EE0083A3F0852A82852983A3A3E0FDE975F0C4
:1055FE0018A424A8FFE5F03480FE8F82F583A3A3C0
:10560E00EDF0852A828C83A3A3A3E08F828E83A3E1
:04561E00A3A3F02230
:065386008D2EAB07AA0604
:10538C00908000E030E507907E547401F022907F0D
:10539C00D3E0FCA3E0FDA3E0FEA3E0F5328E318D5B
:1053AC00308C2FAE02AF038E838F8263A201E53166
:1053BC00540744C0F58385328263A201AF2E123D9F
:1053CC0043E4FCFDFEE532252EF532EE3531F531A8
:1053DC00ED3530F530EC352FF52F908040E52FF082
:1053EC00A3E530F0A3E531F0A3E532F09080007432
:1053FC0020F0AF32AE31AD30AC2F907FD3122C59A0
:01540C00227D
:06540D008D29AB07AA0681
:10541300908002E030E507907E547403F022907F81
:10542300D7E0FCA3E0FDA3E0FEA3E0F52D8E2C8DD9
:105433002B8C2AAE02AF038E838F8263A201E52CED
:10544300540744D0F583852D8263A201AF29123D11
:1054530043E4FCFDFEE52D2529F52DEE352CF52C39
:10546300ED352BF52BEC352AF52A908058E52AF0FB
:10547300A3E52BF0A3E52CF0A3E52DF090800274B7
:1054830020F0AF2DAE2CAD2BAC2A907FD7122C5928
:0154930022F6
:02508F008F2F61
:10509100908001E030E509907E547402F07F002297
:1050A100907FDBE0FCA3E0FDA3E0FEA3E0F5338EFF
:1050B100328D318C30907F5763A201E53254074421
:1050C100C8F58385338263A2017F06123D59E5331A
:1050D1002406F533E43532F532E43531F531E43582
:1050E10030F530907E5563A201E532540744C8F58E
:1050F1008385338263A201AF2F123D59E4FCFDFE8B
:10510100E533252FF533EE3532F532ED3531F53115
:10511100EC3530F53090804CE530F0A3E531F0A36B
:10512100E532F0A3E533F09080017420F0AF33AEA7
:0D51310032AD31AC30907FDB122C59AF2F26
:01513E00224E
:1049E7009081E0E0F52905290529052905290529EB
:1049F70005290529052905290529908010E0F52CA9
:104A0700A3E0F52DA3E0F52EA3E0F52F9081E1E0DB
:104A1700F52905290529052905290529052905292F
:104A2700052905290529908014E0F530A3E0F53123
:104A3700A3E0F532A3E0F533E532B52E08E533B54B
:104A47002F037F0022E4F529E532540744E0F5837C
:104A570085338263A201907C5163A2017F08123DD6
:104A670089907C5363A201907B8963A2017F061220
:104A77003CD1907C51E0F52AA3E0F52BE4F5299091
:104A87007C51E0702AA3E024F8F529E53254074465
:104A9700E0F58385338274082582F582E43583F552
:104AA7008363A201907C5163A201AF29123D89AEB5
:104AB7002AE4FCFDE533252BF533E5323EF532EDEF
:104AC7003531F531EC3530F530908014E530F0A311
:104AD700E531F0A3E532F0A3E533F09080007440B0
:034AE700F0AF2904
:014AEA0022A9
:103F83009081E6E0F5290529052905290529052953
:103F930005290529052905290529908028E0F52CFF
:103FA300A3E0F52DA3E0F52EA3E0F52F9081E7E044
:103FB300F52905290529052905290529052905299E
:103FC30005290529052990802CE0F530A3E0F5317A
:103FD300A3E0F532A3E0F533E4F529E532B52E0A83
:103FE300E533B52F05C22A0240EFE532540744F00A
:103FF300F58385338263A201907C5163A2017F081C
:10400300123D89907C51E0F52AA3E0F52BE52B4581
:104013002A70099080027410F07F0022907F5EE086
:10402300FFF46030907C53E06F60030240B6907FF2
:104033005FE0FF907C54E06F7079907F60E0FF90C9
:104043007C55E06F706D907F61E0FF907C56E06F70
:104053006031805F907C53E0907F5EF0907C54E011
:10406300907F5FF0907C55E0907F60F0907C56E00D
:10407300907F61F0907C57E0FFA3E0907C25CFF028
:10408300A3EFF0907C51E0702AA3E024F8F529E532
:1040930032540744F0F58385338274082582F58210
:1040A300E43583F58363A201907C5163A201AF29B8
:1040B300123D89AE2AE4FCFDE533252BF533E532C9
:1040C3003EF532ED3531F531EC3530F530AF2FAE0D
:1040D3002EAD2DAC2CAB33AA32A931A830D3122C80
:1040E3004840099080027410F07F002290802CE5F4
:1040F30030F0A3E531F0A3E532F0A3E533F090808F
:06410300027440F0AF2938
:014109002293
:104288009081E3E0F529052905290529052905294E
:104298000529052905290529052990801CE0F52C03
:1042A800A3E0F52DA3E0F52EA3E0F52F9081E4E03F
:1042B800F529052905290529052905290529052996
:1042C800052905290529908020E0F530A3E0F5317E
:1042D800A3E0F532A3E0F533E4F529E532B52E0A7B
:1042E800E533B52F05C22B0243DEE532540744E817
:1042F800F58385338263A2019078DF63A2017F0E84
:10430800123D9F9078DFE0F52AA3E0F52B9078E73F
:10431800E0FFF4604A907F57E0FEEF6E7079A3E00B
:10432800FF9078E8E06F706F907F59E0FF9078E930
:10433800E06F7063907F5AE0FF9078EAE06F705703
:10434800907F5BE0FF9078EBE06F704B907F5CE0D4
:10435800FF9078ECE06F703FE49078EEF080089082
:1043680078EE74FFF0D2D99078DFE0702AA3E024C9
:10437800F2F529E532540744E8F583853382740E53
:104388002582F582E43583F58363A2019078DF63A3
:10439800A201AF29123D9FAE2AE4FCFDE533252B8F
:1043A800F533E5323EF532ED3531F531EC3530F5A2
:1043B80030AF2FAE2EAD2DAC2CAB33AA32A931A81D
:1043C80030D3122C485006E52B452A7009908001FD
:1043D8007410F07F0022908020E530F0A3E531F0E2
:1043E800A3E532F0A3E533F09080017440F0AF29E3
:0143F80022A2
:044AEB008E2E8F2F4D
:104AEF00908000E030E507907E547401F022907FB3
:104AFF00D3E0FCA3E0FDA3E0FEA3E0F5358E348DFB
:104B0F00338C32E535FFE5345407FEE42FF531EEF3
:104B1F0034C0F530853182F5837423F00531E531EA
:104B2F00700205305330C7F582853083740AF00563
:104B3F0031E531700205305330C7907C1A63A20102
:104B4F0085308385318263A2017F06123D4374064F
:104B5F002531F531E43530F530852E83852F82638D
:104B6F00A20185308385318263A201123D27E4FCC7
:104B7F00FDFE907FD3E0F8A3E0F9A3E0FAA3E02FC6
:104B8F00FFEE3AFEED39FDEC38FCEF2408FFE43E72
:104B9F00FEE43DFDE43CFC907FD3122C59907FD373
:104BAF00E0908040F0907FD4E0908041F0907FD5EE
:104BBF00E0908042F0907FD6E0908043F0908000AC
:034BCF007420F05F
:014BD20022C0
:0A48E0008E358F368C378D388B39FA
:1048EA00908000E030E507907E547401F022907FBA
:1048FA00D3E0FCA3E0FDA3E0FEA3E0F53F8E3E8DEE
:10490A003D8C3CE53FFFE53E5407FEE42FF53BEEC8
:10491A0034C0F53A853B82F5837423F0053BE53BC9
:10492A007002053A533AC7F582853A83740AF0054C
:10493A003BE53B7002053A533AC7907C1A63A201E1
:10494A00853A83853B8263A2017F06123D43740642
:10495A00253BF53BE4353AF53A853583853682635E
:10496A00A201853A83853B8263A201123D278F40CB
:10497A00EF253BF53BE4353AF53AE53960178537DB
:10498A008385388263A201853A83853B8263A201CB
:10499A00AF39123D43E54024082539F539FFE4FCD7
:1049AA00FDFEE53F2FF53FEE353EF53EED353DF593
:1049BA003DEC353CF53C908040E53CF0A3E53DF00C
:1049CA00A3E53EF0A3E53FF09080007420F0AF3FEE
:0C49DA00AE3EAD3DAC3C907FD3122C599A
:0149E60022AE
:064CB4008E2E8F2F8D30C3
:104CBA00908000E030E507907E547401F022907FE6
:104CCA00D3E0FCA3E0FDA3E0FEA3E0F5368E358D2C
:104CDA00348C33E536FFE5355407FEE42FF532EE22
:104CEA0034C0F531853282F5837423F00532E5321A
:104CFA00700205315331C7F582853183EBF00532F5
:104D0A00E532700205315331C7907C1A63A20185DE
:104D1A00318385328263A2017F06123D43740625E0
:104D2A0032F532E43531F531852E83852F8263A23F
:104D3A000185318385328263A201AF30123D43740B
:104D4A00082530F530FFE4FCFDFEE5362FF536EE9A
:104D5A003535F535ED3534F534EC3533F5339080AA
:104D6A0040E533F0A3E534F0A3E535F0A3E536F0EA
:104D7A009080007420F0AF36AE35AD34AC33907FFE
:044D8A00D3122C59BB
:014D8E002202
:025519008F46BB
:10551B00908000E030E507907E547401F022907F7C
:10552B00D3E0FCA3E0FDA3E0FEA3E0F54A8E498D9A
:10553B00488C47E54AFFE5495407FEE42FFFEE345C
:10554B00C0907B9063A201F5838F8263A201AF466B
:10555B00123D43E4FCFDFEE54A2546F54AEE35498E
:10556B00F549ED3548F548EC3547F547908040E572
:10557B0047F0A3E548F0A3E549F0A3E54AF0908096
:10558B00007420F0AF4AAE49AD48AC47907FD312C0
:02559B002C5989
:01559D0022EB
:064BD3008E298F2AAB05BC
:104BD900908000E030E507907E547401F022907FC8
:104BE900D3E0FCA3E0FDA3E0FEA3E0F5308E2F8D1A
:104BF9002E8C2DE530FFE52F5407FEE42FF52CEE22
:104C090034C0F52B852C82F5837423F0052CE52C13
:104C19007002052B532BC7F582852B83EBF0052CEE
:104C2900E52C7002052B907C1A63A201852B8385E4
:104C39002C8263A2017F06123D437406252CF52CB4
:104C4900E4352BF52B532BC7E529852C82852B833E
:104C5900F0052CE52C7002052B532BC7F582852B0B
:104C690083E52AF0052CE52C7002052B532BC7E5AB
:104C790030240AF530E4352FF52FE4352EF52EE4EE
:104C8900352DF52D908040E52DF0A3E52EF0A3E517
:104C99002FF0A3E530F09080007420F0AF30AE2FF4
:0A4CA900AD2EAC2D907FD3122C59D4
:014CB30022DE
:0A5EF600E4FEEEC39F50030E80F897
:015F0000227E
:10513F00E4F529E5292401FFE433FE125B577412CD
:10514F002529F582E4347CF583EFF00529E529C3A1
:10515F00943F40DFE4F529E529247FFFE433FE1275
:10516F005B5774082529F582E4347AF583EFF074E0
:10517F00082529F582E4347AF583E0FF6003B4FF54
:10518F001D74082529F582E4347AF5837420F074B0
:10519F00092529F582E4347AF583E4F0800905299D
:1051AF00E529C3948040B0E4907A87F0F529AF29C0
:1051BF007E00125B5774882529F582E4347AF583D3
:0B51CF00EFF00529E529C394FE40E342
:0151DA0022B2
:105DB900E4FDFCC3ED9FEC9E5015E4FBFA0BBB0020
:0F5DC900010ABA01F8BB90F50DBD00010C80E492
:015DD80022A8
:0D5ECF004390014390025390FE5390FD223A
:0D5EDC005390FD5390FE439002439001222D
:0E5EB1005390FD439002E5905408FF5390FD7E
:015EBF0022C0
:0D5EE9005390FD4390014390025390FD2221
:075F0C00AE071FEE70FA2240
:025CA400AD074A
:105CA600E4FC5390FDEDA804088002C333D8FC3011
:105CB600E70543900180035390FE7F05125F0C4376
:095CC60090020CBC08DC5390FDB7
:015CCF0022B2
:105D2300E4FF5390FD7E07439002E59030E00D744D
:105D330001A806088002C333D8FC42075390FD1E16
:085D4300C3EE6480948050DF80
:015D4B002235
:105CD000AB05AA07125ECF7FA0125CA4125EB1AF23
:105CE00002125CA4125EB1AF03125CA4125EB11288
:0A5CF0005EDC7F0A7E00125DB9221F
:045B5700AB07AA06E8
:105B5B00C3EB94FFEA9400400DE42BF58274773A83
:105B6B00F583E493FF22125ECF7FA0125CA4125E3A
:105B7B00B1AF03125CA4125EB1125ECF7FA1125CB7
:0D5B8B00A4125EB1125D23125EE9125EDC11
:015B980022EA
:025C0E008B2EDB
:105C1000A2AF9231C2AF85A22F53A2FE8E838F8294
:105C200005A28C838D827409123DCDE52E53A2FE10
:105C300043A220123DCF53A2DF852FA2A23192AF03
:015C4000FF64
:015C41002240
:105DF900A2AF9231C2AF8C838D82EF123DCD43A207
:0C5E090020123DCF53A2DFA23192AFFF68
:015E1500226A
:025D71008F2978
:105D7300A2AF9231C2AFE4F5838D827406123DCD9A
:105D8300E52943A220123DCF53A2DFA23192AF7F78
:015D9300010E
:015D940022EC
:025D95008F2954
:105D9700A2AF9231C2AFE4F5838D82740A123DCD72
:105DA700E52943A220123DCF53A2DFA23192AF7F54
:015DB70001EA
:015DB80022C8
:103BF600A907E7FFA805EF93C3966008403B74FC4E
:103C06002FFF80F00F08EF93C3966008402B74FBDC
:103C16002FFF80E00F08EF93C3966008401B74FAED
:103C26002FFF80D00F08EF93D3966008400B74F9EE
:103C36002FFF80C01F1F1F1F1FEF54FEF80303F73F
:103C4600E893FC08E893FD08E893FE08E893FF2252
:103C560009E993C39D6008402974FB29F980F1099D
:103C6600E993C39E6008401A74FA29F980E209E9CB
:103C760093D39F6008400B74F929F980D319191959
:103C86001919E9C313C313FF22740093F8ECC39800
:103C96004024701F740193F8EDC398401970147492
:0E3CA6000293F8EEC398400E7009740393F871
:103CB400EFC39840037F00227F0122EDF8E6F0086D
:103CC400A3DFFA22EDF8E0F608A3DFFA22E0A3630B
:103CD400A201F0A363A201DFF475A2002263A20192
:103CE400F0A363A20122E0A363A201F0A363A201F3
:103CF400E0A363A201F0A363A201E463A201F0A321
:103D040063A201DFE175A20022E0A363A2016DFEBC
:103D1400936CFDEE058393FC158363A201DFEA75C2
:103D2400A200227F00E493A363A201F00F600CA31E
:103D3400E583C2E3F58363A20180EA75A20022E071
:103D4400A363A201F0A3E583C2E3F58363A201DFC9
:103D5400EE75A20022E0A363A201F0A3E583C2E40E
:103D6400D2E3F58363A201DFEC75A20022E0A36332
:103D7400A201F0A3E58344F8C2E5F58363A201DF61
:103D8400EC75A20022E583C2E3F583E0A363A201FC
:103D9400F0A363A201DFEE75A20022E583C2E4D2A0
:0A3DA400E3F583E0A363A201F0A39E
:103DAE0063A201DFEC75A20022E58344F8F583E0FF
:103DBE00A363A201F0A363A201DFEE75A20022F9B4
:103DCE0022C002C004C00612FFF0D006D004D002FA
:013DDE0022C2
:10090E000A53656E643A20000A43524320657272A0
:10091E006F722120000A53796E63204572726F72D6
:10092E002120000A526563204F4B2120003C2100FC
:10093E0020000ACDE5F220E4EEF1F2EEE2E5F0ED74
:10094E00EEE920E8EDF4EEF0ECE0F6E8E820EFEE6C
:10095E00200020D2D10A0020D2C8D20A000ACAE250
:10096E00E8F220EAEEEDF40A000ACAE2E8F220ED1F
:10097E00E020D2D30A000ACDE5E8E7E2E5F1F2ED98
:10098E00FBE920EFE0EAE5F2202D20000ACFF0E8A7
:10099E00EDFFF220F6E8EAEBE8F7E5F1EAE8E92008
:1009AE00EFE0EAE5F220D2D12000202D20EEF8E88B
:1009BE00E1EAE020E4EBE8EDFB210A00202D20EE39
:1009CE00F8E8E1EAE020EDEEECE5F0E020E1EBEE18
:1009DE00EAE0210A00202D20EEEA210A00202D2037
:1009EE004F7574000ACFF0E8EDFFF220D2D120F15E
:1009FE00EE20E2F0E5ECE5EDE5EC20000ACEF2E2C9
:100A0E00E5F220EDE020E7E0EFF0EEF120D2D30AA0
:100A1E00000AC4E0FE20EAEEECE0EDE4F320E8F19B
:100A2E00EFEEEBEDE8F2FC20D2D30A000AD2D3208F
:100A3E00E8F1EFEEEBEDE5EDEE20F3F1EFE5F8ED9D
:100A4E00EE210A000ACEF2EFF0E0E2EAE020EFEE4D
:100A5E0020F2E0E9ECE0F3F2F3000ACEF2EFF0E080
:100A6E00E2EAE020EFE0EAE5F2E020E8E720EEF748
:100A7E00E5F0E5E4E8003E2A2C312CCFE0F0E0EC86
:100A8E00E5F2F0FB20F1E8EDF5F0EEEDEDEEE3EE44
:100A9E0020EFEEF0F2E00A003E4C2C4230312C25D5
:100AAE006C752CD1EAEEF0EEF1F2FC20EEE1ECE505
:100ABE00EDE02C35302C3130302C3230302C3330C0
:100ACE00302C3630302C313230302C323430302C19
:100ADE00343830300A003E422C4731302C256275B6
:100AEE002CC8EDE2E5F0F1E8FF20EDE020EFF0E8B4
:100AFE00B8ECE50A003E422C4731312C2562752CAC
:100B0E00C8EDE2E5F0F1E8FF20EDE020EFE5F0E5DD
:100B1E00E4E0F7E50A003E422C4730322C256275A0
:100B2E002CD3EFF0E0E2EBE5EDE8E520EFEEF2EEB0
:100B3E00EAEEEC2020285254532D435453290A0038
:100B4E003E532C4730332C256C752CC7E0E4E5F072
:100B5E00E6EAE020F1F2E0F0F2E020EFE5F0E5E485
:100B6E00E0F7E828ECF1290A003E2A2C312CCCEED5
:100B7E00F1F2EEE2EEE920EAEEEDF2F0EEEBEBE56D
:100B8E00F020CACF2022C8F1E5F2FC222E20CFF0B1
:100B9E00EEF2EEEAEEEB2022C3F0E0EDE8F22220D8
:100BAE002D20F1E8EDF5F0EEEDEDFBE92C2000EA5D
:100BBE00EBE0F1F1E8F7E5F1EAE8E92E0A00F0E002
:100BCE00F1F8E8F0E5EDEDFBE92E0A003E422C4788
:100BDE0030312C2562752CD0E0F1F8E8F0E5EDED22
:100BEE00FBE920EFF0EEF2EEEAEEEB0A003E532CBC
:100BFE004730342C2562752CCDEEECE5F020CACFB3
:100C0E000A003E432C4731392C25732CCAEEEDF4E5
:100C1E00E8E3F3F0E0F6E8FF20CACF3A0A00202519
:100C2E0062752020202562752020202025627520E7
:100C3E00202025627520003E532C4731382C257319
:100C4E002CF1F2E0F0F2EEE2FBE520EDEEECE5F059
:100C5E00E020C0D4C13A0A003E422C4730352C2544
:100C6E0062752CCCE0E3E8F1F2F0E0EBFCEDFBE991
:100C7E0020F0E5E6E8EC0A003E422C4730362C2503
:100C8E0062752CD2D120EFEE20E7E0EFF0EEF1F31B
:100C9E000A003E422C4730372C2562752CD2C8D222
:100CAE0020EFEE20E7E0EFF0EEF1F30A003E532CDA
:100CBE004730382C2562752CD2E0E9ECE0F3F220B7
:100CCE00EFE5F0E5F5EEE4E020EA20E8EDE8F6E801
:100CDE00E0F2E8E2EDEEE920EFE5F0E5E4E0F7E53D
:100CEE002863290A003E4C2C4730392C256C752C74
:100CFE00CAEEEDF42E20D2D32C3136202D20EFF07B
:100D0E00FFECEEE520F3EFF02E2C3330202D20F10A
:100D1E0020E8F1EF2E20F0E5EBE52C313238202DD6
:100D2E0020C1D0CF20C3F0E0EDE8F20A003E422C05
:100D3E004731342C2562752C2B20ECE5E0EDE4F0E8
:100D4E0020EFE5F0E5E420EEF2EAF0FBE2E0FEF95A
:100D5E00E8EC20F4EBE0E3EEEC0A003E422C4732E6
:100D6E00312C2562752CC1EBEEEAE8F0EEE2E0F2F2
:100D7E00FC20D2D120F120ECE5F2EAE0ECE820E212
:100D8E00F0E5ECE5EDE80A003E422C4731352C2526
:100D9E0062752CCFE5F0E5E4E0E2E0F2FC20E0F055
:100DAE00F5E8E220D2D120EFF0E820F1F2E0F0F207
:100DBE00E50A003E422C4732352C2562752CD2C8EE
:100DCE00D220EAE0EA20E220D1E8F1F2E5EB0A00D7
:100DDE003E532C4731372C25732CD0E5E2E5F0F14C
:100DEE00E8E2EDFBE520D2C8D20A003C4230313DAC
:100DFE00003C4731303D003C4731313D003C4730EF
:100E0E00323D003C4730333D003C4730313D003CE5
:100E1E004730343D003C4730353D003C4730363D91
:100E2E00003C4730373D003C4730383D003C4730B2
:100E3E00393D003C4731353D003C4732353D003CA5
:100E4E004731343D003C4732313D003C4731373D60
:100E5E00000008040C020A060E0109050D030B071B
:100E6E000F00112332465765748C9DAFBECADBE965
:100E7E00F810013322564775649C8DBFAEDACBF95C
:100E8E00E82130021367764455ADBC8E9FEBFAC84D
:100E9E00D93120120377665445BDAC9E8FFBEAD83C
:100EAE00C94253617004152736CEDFEDFC8899AB2D
:100EBE00BA5243716014053726DECFFDEC9889BB1C
:100ECE00AA6372405125340617EFFECCDDA9B88A0D
:100EDE009B7362504135241607FFEEDCCDB9A89AFC
:100EEE008B8495A7B6C2D3E1F008192B3A4E5F6DED
:100EFE007C9485B7A6D2C3F1E018093B2A5E4F7DDC
:100F0E006CA5B48697E3F2C0D129380A1B6F7E4CCC
:100F1E005DB5A49687F3E2D0C139281A0B7F6E5CBB
:100F2E004DC6D7E5F48091A3B24A5B69780C1D2FAC
:100F3E003ED6C7F5E49081B3A25A4B79681C0D3F9B
:100F4E002EE7F6C4D5A1B082936B7A48592D3C0E8C
:100F5E001FF7E6D4C5B1A092837B6A58493D2C1E7B
:100F6E000F0089129B24AD36BF48C15AD36CE57E63
:100F7E00F78108931AA52CB73EC940DB52ED64FFEA
:100F8E0076028B109926AF34BD4AC358D16EE77CDA
:100F9E00F5830A9118A72EB53CCB42D950EF66FDCA
:100FAE0074048D169F20A932BB4CC55ED768E17ABA
:100FBE00F3850C971EA128B33ACD44DF56E960FBAA
:100FCE0072068F149D22AB30B94EC75CD56AE3789A
:100FDE00F1870E951CA32AB138CF46DD54EB62F98A
:100FEE007008811A932CA53EB740C952DB64ED768A
:100FFE00FF89009B12AD24BF36C148D35AE56CF76A
:10100E007E0A8318912EA73CB542CB50D966EF7459
:10101E00FD8B029910AF26BD34C34AD158E76EF549
:10102E007C0C851E9728A13AB344CD56DF60E97239
:10103E00FB8D049F16A920BB32C54CD75EE168F329
:10104E007A0E871C952AA338B146CF54DD62EB7019
:10105E00F98F069D14AB22B930C74ED55CE36AF109
:0F106E0078D2D120D2C8D220D2D320D2C8C80085
:105D000052600000000000000000000000000000E1
:105D100000000000004A646900000000000000006C
:025D2000000081
:105DD900906FBFE06FFC900F6F93FE906FBCE06E09
:0F5DE900906FBFF0AF04EF900E6F93906FBCF010
:015DF8002288
:10001E00EF540F900E5F93FEC454F0FEEFC4540FD6
:04002E00932EFF22EC
:105C420030202CE4907D51F0E57C24FEFFA3F090FF
:105C52007F56E0907D53F0A37408F0906E3D63A2EE
:105C620001907D5563A201123CD1C2207F01227FA7
:025C720000220E
:1059A200C231E4FEE57A64056032BF7E07D206E4C6
:1059B200F575F57AEF30E707436B01057A800653F8
:1059C2006BFEE4F57A0575E575B40808856B7FD240
:1059D20031E4F575E56B25E0F56B800CEF30E705FA
:1059E200D206A23122E4F57AEF25E0FF0EBE08B41A
:0259F200A231E0
:0159F4002290
:10570A00E4FEE57425E0F574EF30E73643740120D2
:10571A0032330573E573B4052CE4F5730579E5793D
:10572A00B408170571E571AC707002057014F58242
:10573A008C83E574F0057DE4F579E57425E0F5746C
:10574A008003E4F5730579E579B408170571E57105
:10575A00AC707002057014F5828C83E574F0057DD7
:0D576A00E4F579EF25E0FF0EEE6408709580
:01577700220F
:0447D1008E338F3460
:1047D500906FBCE0907F6EF0906FBFE0907F6FF0C0
:1047E500E4F57DF573906FBCF0906FBFF0AB34AA24
:1047F5003375706E7571CD30142585718285708322
:10480500740AF00571E57170020570F58285708393
:1048150074AAF00571E57170020570057D057D8549
:104825007182857083747EF00571E5717002057083
:10483500057DE4F579907F6CF0907F6CE0C39D5029
:104845004B8B828A83E0FF12001E907F6DEFF09004
:104855006FBFE06F907F6DF0E0FF900F6F93FE905C
:104865006FBCE06E906FBFF0EF900E6F93906FBCD2
:10487500F00BEBAE0270010A14F5828E83E0FFC2E5
:104885003212570A907F6CE004F080AD906FBFE064
:10489500FF12001EC23212570A906FBCE0FF1200D1
:1048A5001EC23212570AD2327F7E12570AD232E422
:1048B500FF12570AD2037C6E7DCD8C708D71302F1F
:1048C500097E097F0EAB7D1248E0907F6EE0906F08
:0A48D500BCF0907F6FE0906FBFF021
:0148DF0022B6
:0100320022AB
:104F2700E4FF0F24E0F582E43479F5837408F00F89
:104F370074E02401F582E43479F583E4F07C607D44
:104F470005FEED1DAA0470011CF5828A83E0FBAA09
:104F5700070F74E02AF582E43479F583EBF00EBE8F
:104F670004E07C607D09E4FEED1DAA0470011CF5D8
:104F7700828A83E0FBAA070F74E02AF582E434797A
:104F8700F583EBF00EBE04E07C607D0DE4FEED1DC5
:104F9700AA0470011CF5828A83E0FBAA070F74E05C
:104FA7002AF582E43479F583EBF00EBE04E07C60E9
:104FB7007D11E4FEED1DAA0470011CF5828A83E0D1
:104FC700FBAA070F74E02AF582E43479F583EBF046
:044FD7000EBE04E026
:014FDB0022B3
:105E4D00D209E4F57CF57A906FBFF0906FBCF0F558
:085E5D0075756D6E756E3D2236
:10454C00200903024664E565543865607003024631
:10455C009BE56024085438F560131313541F245042
:10456C00F8E6F57820063020082DFF1259A250D617
:10457C00AF7F12001E125DD9056EE56EAE6D700236
:10458C00056D14F5828E83E57FF0057CE57CD39474
:10459C004040B3D20880AFE57CD39402400520089C
:1045AC0002D220C209C206E4F54ED23A906FBFE0A7
:1045BC00FF906FBCE04F6047C220302F0D7E097F0B
:1045CC00167C6E7D3DAB7C1248E090600AE0FCA34B
:1045DC00E0FDA3E0FEA3E0FFE4FAF9F8EF2401FF0D
:1045EC00EA3EFEE93DFDE83CFC90600A122C599035
:1045FC006E3DE0705E20085BC23A125E4D805490B6
:10460C006E3DE07014C220302F497E097F237C6EF2
:10461C007D3DAB7C1248E0803A302F0D7E097F3116
:10462C007C6E7D3DAB7C1248E0906002E0FCA3E028
:10463C00FDA3E0FEA3E0FFE4FAF9F8EF2401FFEAA2
:10464C003EFEE93DFDE83CFC906002122C59E490E2
:10465C0078C1F0C208024552203A34E550B47E0FBE
:10466C00300408E4F54ED23AC20422125E4D22E523
:10467C0050B56716200713D20190601CE0FFA3E031
:10468C009065F8CFF0A3EFF0C20AE4F54ED23A22CF
:0B5F0100301F05C21F7F01227F00221D
:104FDC009078D974FFF0A374B8F0E49078D8F0907E
:104FEC0078C504F09064737410F0C207C20FC20D40
:104FFC00D20BC20CC21190601C7402F0A374EEF0C0
:10500C00123467300B07906F7AE0B4010E90601A7F
:10501C007410F09060177402F0800C90601A740891
:10502C00F09060177404F0E4906051F0906018F008
:10503C00C215C21AC216C217D21ED21D906FBEF074
:10504C00907F6BF0907F6BE0FFC394085018EF25B6
:10505C00E024BDF582E4346EF583E4F0A3F0907F98
:10506C006BE004F080DE9078C37402F0A37471F0EE
:10507C0090601CE0FFA3E09065F8CFF0A3EFF01276
:02508C0057D9F2
:01508E0022FF
:015F1300226B
:102D3600756A7E3007047F5580027FA08F67C209BF
:102D4600D213C220D23AC21CC203C21FD201C2177A
:102D5600E4906E3CF09078C6F0907F6BF0907F6BBD
:102D6600E0FFC3947F501975F009EFA424C0F582E3
:102D7600E5F0346FF583E4F0907F6BE004F080DDDE
:102D8600E4906016F0906F4D7464F0E49065FAF08C
:102D9600A3F0906012F0A3F0A3F0A3F0906F7BF085
:102DA60090601BF07B0190647404F0A3746FF0A331
:102DB600747CF090604EEBF0A37461F0A37468F03D
:102DC600E4907F74F0A3F0A3F0A304F0907F76E084
:102DD600FCA3E0FDC39405EC94004003022E7A9018
:102DE6007F75E0C4F8540FC868FF907F74E0C45440
:102DF600F0487E00EF5430FFED2FFFEE3C907F70E1
:102E0600F0A3EFF0E4907F6EF0A3F0907F71E0FF07
:102E1600906474E0FBA3E0FAA3E0F9EF122999901D
:102E26006474E0FBA3E0FAA3E0F9900001E4122940
:102E3600AB906475E475F002122A58907F6FE00437
:102E4600F07006907F6EE004F0907F6EE07004A351
:102E5600E0640870B6907F77E004F07006907F76A5
:102E6600E004F0907F75E004F07006907F74E00453
:102E7600F0022DD2E4907F6BF07E097F3B125494D2
:102E8600EF4E7021907F6BE0FF90780093FE7452B6
:102E96002FF582E43460F583EEF0907F6BE004F06A
:102EA600E070E18019907F6BE02452F582E4346093
:102EB600F5837401F0907F6BE004F0E070E7E49036
:102EC6007F6DF0907F6CF0907F6BF0907F6BE024CD
:102ED60077F582E43464F583E0FF7003022FC9902E
:102EE6007F6CE0C3748094814003022FC9EFB42045
:102EF60008907F6BE004F080D2907F6BE02477F53A
:102F060082E43464F583E0642D7037907F6BE004CF
:102F1600F0E02477F9E43464FA7B01C0031B8B31BB
:102F2600753200753300E4F534D003123DDF907F2F
:102F36006DEFF0907F6CE0FEC3EF9EA3F0E004F02F
:102F46008029907F6BE02477F9E43464FA7B01C032
:102F5600031B8B31753200753300E4F534D0031250
:102F66003DDF907F6CEFF0A37401F0907F6DE0D3AE
:102F760094004023907F6CE0FF7480948150187415
:102F8600512FF582E43460F583E4F0907F6CE00421
:102F9600F0A3E014F080D4907F6BE02477F582E410
:102FA6003464F583E0FF64207003022ED1EF642DB4
:102FB6007003022ED1EF7003022ED1907F6BE004D6
:102FC600F080D4E4907F6BF0907F72F0A3F0907F56
:102FD60076F0A37405F0E4907F74F0A3F090601788
:102FE600E0FFC3907F75E09F907F74E094004003FC
:102FF6000230EA907F73E0C4F8540FC868FF907FF0
:1030060072E0C454F0485401FEEF54F0FF907F770D
:10301600E02FFF907F76E03E907F70F0A3EFF0E424
:10302600907F6EF0A3F090601AE0FFC3907F6FE090
:103036009F907F6EE0940040030230CB200B3F90C0
:103046007F6BE0FF04F074522FF582E43460F58361
:10305600E07010907F71E02400FF907F70E03420D4
:10306600FE8008907F70E0FEA3E0FF90604EE0FBDC
:10307600A3E0FAA3E0F9EE8FF0122AD18018907F30
:1030860070E0F9A3E0FF90604EE0FBA3E0FAA3E056
:10309600C98FF0122AD190604EE0FBA3E0FAA3E0BC
:1030A600F9900002E4F5F0122AF090604FE475F012
:1030B60004122A58907F6FE004F07006907F6EE04D
:1030C60004F002302C907F75E004F07006907F7457
:1030D600E004F0907F73E004F07006907F72E004E5
:1030E600F0022FE3907F77E004F07006907F76E0A1
:1030F60004F0907F76E07004A3E0640B6003022F77
:04310600DC125EC0B9
:01310A0022A2
:105E1600907E557444F0A37418F0A3EDF0A3EFF050
:0D5E2600A37401F0E4A3F07F0612508F2258
:1043F90075F008EFA4243CF582E5F03466AF82F548
:104409002E8F2FF583A3A3A3E0FF852F82852E830B
:10441900A3A3E02FFFE433FEE52F2404F582E4355E
:104429002EF583E07C002FFFEC3EFEE52F2405F5F9
:1044390082E4352EF583E02FFFEC3E4F7002FF2218
:104449009078C5E0906F4EF0906FBEE024F0906FC9
:104459004FF0906FBEE004F0540FF0906F50740667
:10446900F0A37491F0906014E0FEA3E0906F52F015
:10447900EEA3F0302F0D7E097F3E7C607D147B0218
:104489001248E0852F82852E83A3A3E0906F54F014
:10449900852F82852E83A3A3A3E0906F55F0E52F86
:1044A9002404F582E4352EF583E0906F56F0E52F6C
:1044B9002405F582E4352EF583E0906F57F0852FBA
:1044C90082852E83A3E0FB540FFEC454F0FE852F92
:1044D90082852E83E0FDC313042E906F58F0ED54AE
:1044E90003FF25E0FFEB5410FEC4540F2FA3F0E5A2
:1044F9002F2407F582E4352EF583E0FEE52F240607
:10450900F582E4352EF583E07C002400FFEC3EFEC5
:104519007D0A1229CDEF547F906F5AF0852F82853D
:104529002E83A3E030E709906F5AE04480F08007BA
:10453900906F5AE0547FF07E6F7F4E7D0D1247D108
:024549007F01F0
:01454B00224D
:024E5C00AB07A2
:104E5E0075F009EFA424C0F582E5F0346FAD82FC45
:104E6E00F583E054BFF00DBD00010C9078C5E090C5
:104E7E006F4EF0906FBEE024F0906F4FF0906FBECB
:104E8E00E004F0540FF0906F507403F0A37491F09F
:104E9E00EBC4540F240CA3F0EB540FA3F08D828CB3
:104EAE0083E0906F59F00DBD00010C8D828C83E074
:104EBE00906F5AF00DBD00010C8D828C83E0906FC7
:104ECE005BF00DBD00010C8D828C83E0906F5CF069
:104EDE000DBD00010C8D828C83E0906F54F00DBDE2
:104EEE0000010C8D828C83E0906F55F00DBD00019A
:104EFE000C8D828C83E0906F56F00DBD00010CAED0
:104F0E0004AF058F828E83E0906F57F0E4A3F07E9E
:084F1E006F7F4E7D0F1247D199
:014F26002268
:1059F5008F2E9078C5E0906F4EF0E52E24A0A3F091
:105A0500E4A3F0A37402F07E6F7F4E7D041247D1AC
:105A1500302F277E097F40E4FBFDFC1248E0E52E90
:105A2500B4080C7E097F60E4FBFDFC1248E0227E91
:0B5A3500097F65E4FBFDFC1248E02245
:105C74009078C5E0906F4EF0E57B24F0A3F0A37418
:105C8400FEF0A3748FF07E6F7F4E7D041247D1C265
:105C94000E302F0B7E097F6BE4FBFDFC1248E022E3
:105A89009078C5E0906F4EF0907F6B740BF0906446
:105A9900F7E0D394074006907F6BE004F0907F6BAA
:105AA900E02480906F4FF0E4A3F0A3F07E6F7F4E67
:105AB9007D041247D1C202302F0B7E097F77E4FBA8
:055AC900FDFC1248E0A5
:015ACE0022B5
:105E65009078C5E0906F4EF0A37490F07E6F7F4EF2
:065E75007D021247D1225C
:105D4C00300A099065F8E4F0A37414F0906ECD74E9
:105D5C00AAF0A374A0F0E4A3F0D20375706E757171
:055D6C00CD757D03224E
:10526B00E4907F6BF09078C5E0906F4EF0906FBE3E
:10527B00E024F0906F4FF0906FBEE004F0540FF00D
:10528B00E4906F50F0A37490F0A37408F0E4A3F0D3
:10529B00906F79E0906F54F0906F78E0906F55F0CD
:1052AB00906F77E0906F56F0906F76E0906F57F0BD
:1052BB00C37464956CA3F0907F6B740BF0907F6B51
:1052CB00E0FFC3940F5014744E2FF582E4346FF546
:1052DB0083E4F0907F6BE004F080E27E6F7F4E7D85
:0E52EB000F1247D19078C37407F0A37453F0EC
:0152F9002292
:02107D00AB07BF
:10107F00301E0B9078C3E4F0A37414F0C21E907866
:10108F00DFE024BE700302170724FE601B24FC70F0
:10109F00030215A08000202F0302179C7E097F8476
:1010AF007C787DDF1248E0229078E0E054E324DF83
:1010BF0070030212AB24A170030213362460600385
:1010CF0002179C9078E2E0600302179C9078E9E0A9
:1010DF00FE9078E8E07C002400FFEC3E907F6BF000
:1010EF00A3EFF0302F0D7E097F9A7C7F7D6B7B0203
:1010FF001248E09078E3E064066012202F03021795
:10110F009C7E097FB8E4FBFDFC1248E0229078E159
:10111F00E0D394074012202F0302179C7E097FCA49
:10112F00E4FBFDFC1248E0229078E1E0FE540790CA
:10113F007F6DF0EE25E025E0F52975F002A4247C03
:10114F00F9746F35F0FA9064747401F0A3EAF0A3A8
:10115F00E9F0E4F52A906474E0FBA3E0FAA3E0F968
:10116F0090000112296CFF12001E74E4252AF582EB
:10117F00E43478F583E06F6015906474E0FBA3E0CE
:10118F00FAA3E0F91229534440122999D216906418
:10119F0074E0FBA3E0FAA3E0F9122953448012296B
:1011AF0099906474E0FBA3E0FAA3E0F91229535479
:1011BF000F24C7F582E43478F58374C8F074E425FE
:1011CF002AF582E43478F583E0FF12001E906474F0
:1011DF00E0FBA3E0FAA3E0F9900001EF1229AB9036
:1011EF006475E475F002122A58052AE52AC394049F
:1011FF005003021164907F6DE025E024BDF582E479
:10120F00346EF583E0FEA3E0FF907F6BE0FCA3E07C
:10121F00FDEF6D7002EE6C6071C3EF9DEE9C505050
:10122F0030004D300B4AC3ED9FFFEC9EFED3EF9481
:10123F001EEE9400501EA3E0FD25E024BDF582E4D0
:10124F00346EF583E0FEA3E024FFFFEE34FFFE12C1
:10125F005E168036907F6BE0FEA3E0FFA3E025E0F3
:10126F0024BDF582E4346EF583EEF0A3EFF0801A1F
:10127F00907F6BE0FEA3E0FFA3E025E024BDF582A5
:10128F00E4346EF583EEF0A3EFF0202F0302179CEA
:10129F007E097FE3E4FBFDFC1248E0229078E1E059
:1012AF00FFB56F09A3E06572700302179C9078E396
:1012BF00E06408600302179C8F6F9078E2E0F5728C
:1012CF00EF75F002A4240BFFE435F0FED3EF940F7B
:1012DF00EE64809480400C7E097FEBE4FBFDFC12F2
:1012EF0048E0229078E2E014FF9078E1E0C43354B4
:1012FF00E02FF52975F009A424C0F582E5F0346FCD
:10130F00F583E04440F0D2159078E463A20175F0C4
:10131F0009E529A424C1F582E5F0346FF58363A2B2
:10132F00017F08123CD1229078E3E0640860030249
:10133F00179C9078E1E0FFD39407400302179CEFCE
:10134F005407FF907F6DF0FD9078EBE0FE9078EA08
:10135F00E07A002400FFEA3EFE907F6BF0A3EFF0EF
:10136F00ED25E024BDF582E4346EF583E0FCA3E0C7
:10137F00FD2401FBE43CFAEB6F7002EA6E7003028E
:10138F00142B907F6BE0FAA3E0FBC3ED9BEC9A501C
:10139F004A300B47A3E025E024BDF582E4346EF517
:1013AF0083E0FEA3E0FFC3EB9FFDEA9EFCD3ED9429
:1013BF001EEC94005009907F6DE0FD125E16229096
:1013CF007F6BE0FEA3E0FFA3E025E024BDF582E400
:1013DF00346EF583EEF0A3EFF08041907F6DE0FF68
:1013EF0025E024BDF582E4346EF583E0FCA3E0FD37
:1013FF00907F6BE0FAA3E0FBC3ED9BFDEC9AFCD36F
:10140F00ED941EEC9400500302179CEF25E024BDD1
:10141F00F582E4346EF583EAF0A3EBF0302F0D7E06
:10142F00097FF27C7F7D6B7B021248E0907F6DE03D
:10143F0025E024BDF582E4346EF583E475F00112E6
:10144F002A589078E2E0547FFF131313541FFF9034
:10145F0078E1E025E025E02FF52975F002A4247C42
:10146F00F9746F35F0FA9064747401F0A3EAF0A385
:10147F00E9F09078E2E05407F529752A806010E5CD
:10148F0029D394004009E52A13F52A152980F090F5
:10149F0078E2E030E71A906474E0FBA3E0FAA3E08F
:1014AF002401F9E43AFA122953452A122999801B8B
:1014BF00906474E0FBA3E0FAA3E02401F9E43AFAA4
:1014CF00122953FFE52AF45F122999906474E0FB07
:1014DF00A3E0FAA3E0F9122953FF540F24C7F582B2
:1014EF00E43478F58374C8F0EF44C0122999300BB7
:1014FF0003301B03D2162290601BE075F008A42462
:10150F003CF582E5F03466AF82FE9078E1E08F82A1
:10151F008E83F00FBF00010E9078E2E08F828E83F2
:10152F00F00FBF00010E9078E4E08F828E83F00FF2
:10153F00BF00010E9078E5E08F828E83F00FBF0021
:10154F00010E9078E6E08F828E83F00FBF00010EC0
:10155F009078E7E08F828E83F00FBF00010E9078B6
:10156F00E8E08F828E83F00FBF00010E9078E9E0E4
:10157F008F828E83F090601BE004F0301703021708
:10158F009CE49065FAF0A3F0D217906FBD7403F04E
:10159F00229078E2E0FF30E60302179C9078E1E0BA
:1015AF00FEC39406400302179C752D78752EE4EF49
:1015BF00547FFFEEC43354E02FF52975F004A424B3
:1015CF0068F9746135F0FA90604E7401F0A3EAF097
:1015DF00A3E9F09078E3E0FFC313F529E4F52AE5DA
:1015EF002AC39529400302179C300B0302168885E6
:1015FF002E82852D83E0752B00F52CA3E0FEE425CC
:10160F002CF52CEE352BF52B90604EE0FBA3E0FA7A
:10161F00A3E0F9122A6EE5F030E53AC3E52C947891
:10162F00E52B6480946C5006752BEC752C78E52CAB
:10163F002488FFE52B3413FE7C007D28122A22908C
:10164F00604EE0FBA3E0FAA3E0F9900002EE8FF00A
:10165F00122AF08043AF2CAE2B125E8F7C007D14CC
:10166F00122A2290604EE0FBA3E0FAA3E0F990006B
:10167F0002EE8FF0122AF0801F852E82852D83E0D7
:10168F00FEA3E0FF90604EE0FBA3E0FAA3E0F99029
:10169F000002EE8FF0122AF07402252EF52EE4359B
:1016AF002DF52D200F1890604EE0FBA3E0FAA3E07C
:1016BF00F9122A6EFFE5F044408FF0122AD1D21AA8
:1016CF0090604EE0FBA3E0FAA3E0F9122A6EFFAEA2
:1016DF00F07C00540F24C7F582EC3478F58374C87E
:1016EF00F0EE44808FF0122AD190604FE475F00431
:1016FF00122A58052A0215EE9078E2E0640370650D
:10170F009078C6E0605F302F0B7E0A7F0AE4FBFD06
:10171F00FC1248E09064F7E0FF9078E1E06F7040D2
:10172F009078C2E0FF9078E4E06F7034907E55744B
:10173F0002F0A37408F09064F7E0907E57F0A3F0E6
:10174F00A37401F0E4A3F07F0612508F906E3C74E7
:10175F0020F0302F0B7E0A7F1FE4FBFDFC1248E0C8
:10176F00E49078C6F09078E2E064017020906E3CCF
:10177F00E0601A9078E5E07002D202E4906E3CF0DF
:0D178F00302F0A7E0A7F3AFBFDFC1248E075
:01179C00222A
:105B9900906016E0FFC3947F502A75F009EFA424A2
:105BA900C0F582E5F0346FF583E030E60F906016BA
:105BB900E0124E5C906016E004F0D322906016E08B
:0D5BC90004F080CCE4906016F0C215C322F9
:10469C00906F4DE06002C322C231906051E0FF6028
:1046AC0002D2318F2EE52EC3942040030247C6E57B
:1046BC002E131313541FF52FE52E75F002A4247C32
:1046CC00F9746F35F0FA7B01906474EBF0A3EAF0A7
:1046DC00A3E9F012295320E6030247C1E52E540743
:1046EC00FFC3E52E9FF52E2408906051F0E52E7542
:1046FC00F002A4247CF9746F35F0FA906474EBF03A
:10470C00A3EAF0A3E9F07E607F1E9078C5E08F826B
:10471C008E83F00FBF00010E122953FD540F24405D
:10472C008F828E83F00FBF00010EEDC45403242042
:10473C008F828E83F00FBF00010EE4F52E9064740F
:10474C00E0FBA3E0FAA3E0F990000112296C8F8240
:10475C008E83F012295354BF12299974082FFFE449
:10476C003EFE906474E0FBA3E0FAA3E0F990000134
:10477C0012296CF48F828E83F074F82FFF74FF3E35
:10478C00FE906475E475F002122A580FBF00010EFA
:10479C00052EE52EB408A67E607F1E7D131247D130
:1047AC00E52F25E02469F582E43464F583E4F0A375
:1047BC00747DF0D322052E0246B1E4906051F0A234
:0447CC00319216C34D
:0147D00022C6
:10373F00906017E0FF90601AE08FF0A475F006A478
:10374F00F532906018E0F530E530C3953240030252
:10375F0039DF90601AE0FFE5308FF084F531E53006
:10376F0075F004A42468F9746135F0FA7B01906058
:10377F004EEBF0A3EAF0A3E9F0122A6EE5F020E693
:10378F00030239DA90601AE0FFE5308FF084C3E569
:10379F003095F0F5302F906018F0E53075F004A4F7
:1037AF002468F9746135F0FA90604EEBF0A3EAF0FB
:1037BF00A3E9F0906F7AE0B401067E607F1E80046B
:1037CF007E607F1F8E2E8F2F9078C5E0852F82858C
:1037DF002E83F0052FE52F7002052E300B030238D4
:1037EF008890604EE0FBA3E0FAA3E0F9122A6EFF87
:1037FF00AEF0540F2440852F82852E83F0052FE5E0
:10380F002F7002052EEEC4F854F0C868EFC4540FA1
:10381F0048541F2460852F82852E83F0052FE52FB6
:10382F007002052EE4F53090601AE0FFE530C39F7B
:10383F00503B90604EE0FBA3E0FAA3E0F99000024A
:10384F00122A99852F82852E83F0122A6EFFE5F0BA
:10385F0054BF8FF0122AD190604FE475F004122AF2
:10386F0058052FE52F7002052E053080BA7E607F38
:10387F001F7D131247D10239D8906F7AE06401701F
:10388F004A852F82852E837470F0052FE52F7002E5
:10389F00052EF582852E837442F0052FE52F7002D9
:1038AF00052E90604EE0FBA3E0FAA3E0F9122A6E1A
:1038BF00FFE5F0C4F854F0C868EFC4540F48540F34
:1038CF002460852F82852E83F08076906FBEE02452
:1038DF00F0852F82852E83F0906FBEE004F0540F99
:1038EF00F0052FE52F7002052EF582852E837402C9
:1038FF00F0052FE52F7002052EF582852E8374912A
:10390F00F0052FE52F7002052E90604EE0FBA3E02F
:10391F00FAA3E0F9122A6EFDACF0ECC4F854F0C82B
:10392F0068EDC4540F48540FFBEDC4F8540FC8682A
:10393F00FFECC454F048EF54F02B852F82852E8373
:10394F00F0906F7AE0B401067E607F2280047E6083
:10395F007F24E4F53090601AE0FDE530C39D503EC2
:10396F0090604EE0FBA3E0FAA3E0F9900002122A68
:10397F0099FD8F828E83E5F0F0A3EDF0122A6EFD94
:10398F00E5F054BF8DF0122AD190604FE475F0042A
:10399F00122A5874022FFFE43EFE053080B7906F55
:1039AF007AE0FFB401067C607D1E80047C607D1F81
:1039BF008C2E8D2FEFB401047F2480027F158F3062
:1039CF00AD30AF2FAE2E1247D1D32205300237576D
:0839DF00E4906018F0C21AC365
:0139E70022BD
:10577800D218906F4DE07058E4F52EE52EC39420B2
:10578800503FE52E75F002A4247CF9746F35F0FAC9
:105798007B01906474EBF0A3EAF0A3E9F0122953BB
:1057A800FF30E715906474E0FBA3E0FAA3E0F9EF9B
:1057B8004440122999D216C2187404252EF52E8059
:1057C800BA30180C906F76122C6500000000D21EBB
:0157D80022AE
:105ACF00906F7BE075F008A4243EF582E5F0346614
:105ADF00AF82FEF583E4F00FBF00010E8F828E833D
:105AEF00E4F00FBF00010E8F828E83E4F00FBF0032
:105AFF00010E8F828E83E4F00FBF00010E906F7B3B
:035B0F00E004F0BF
:015B12002270
:10179D0030122DC3E54D9569FFE54C9568FED3EFED
:1017AD009440EE940040197B087D40AF69AE6812FD
:1017BD004CB4E5692440FFE43568540FF5688F6932
:1017CD00301D05122D36C21D12454C202203021864
:1017DD00E9C222906F4DE0600214F0E4F52974C760
:1017ED002529F582E43478F583E070030218DE7460
:1017FD00C72529F582E43478F583E014F074C72504
:10180D0029F582E43478F583E060030218DEE529DA
:10181D00D394045048E52975F010A4246CF9746F25
:10182D0035F0FA9064747401F0A3EAF0A3E9F0E4E2
:10183D00F52AE52AC3940840030218DE906474E08B
:10184D00FBA3E0FAA3E0F9122953547F122999055D
:10185D002A906475E475F002122A5880D5E5292482
:10186D00FBFF90601AE0FEEF8EF0A4FF906017E092
:10187D00FEEF8EF0A475F004A42468F9746135F0C0
:10188D00FA90604E7401F0A3EAF0A3E9F0E4F52AB2
:10189D00906017E0FF90601AE08FF0A4FFC3E52A77
:1018AD009FE5F06480F8748098502690604EE0FBC0
:1018BD00A3E0FAA3E0F9122A6EFFE5F0547F8FF052
:1018CD00122AD1052A90604FE475F004122A58802F
:1018DD00BF0529E529641060030217EB20300302D0
:1018ED0019C7C2309078C6E0600214F0906E3CE0EB
:1018FD00600214F09078C3E07002A3E0600E90785F
:10190D00C4E024FFF09078C3E034FFF09065FAE076
:10191D007002A3E0600E9065FBE024FFF09065FA85
:10192D00E034FFF09065F8E07002A3E0603590655B
:10193D00F9E024FFF09065F8E034FFF0E07002A3C9
:10194D00E07020200702D201200A08E49078D7F039
:10195D00125778D20A302F0B7E0A7F52E4FBFDFC22
:10196D001248E0E4F529E52925E02469F582E434FF
:10197D0064F583E0FEA3E04E6037E52925E0246998
:10198D00F582E43464F58374FFF5F0122A58E529E5
:10199D0025E02469F582E43464F583E0FEA3E04E8E
:1019AD00700F300A0C200D099078D77402F0125781
:1019BD00780529E529C3940440AC302435C2249020
:1019CD006468E0600214F0D56C28756C64906F76D5
:1019DD00E0FCA3E0FDA3E0FEA3E0FFE4FAF9F8EFDD
:1019ED002401FFEA3EFEE93DFDE83CFC906F7612D6
:1019FD002C59202003021D0FC2209078C5E0FF90C6
:101A0D006E3DE06F6003021D04A3E0FF54F024F06F
:101A1D00603624E07003021BD724407003021BF0D4
:101A2D0024F06003021D0FEF540FF52BD3940440E7
:101A3D0003021D0FE52B25E02467F582E43464F5E0
:101A4D0083E4F0A3F0021D0F906E3EE0540F14706E
:101A5D0003021AE4147003021AE424F960120460FC
:101A6D0003021D0F9078D77401F0125778021D0FE5
:101A7D00D210906017E0FF90601AE08FF0A475F01F
:101A8D0006A4F52AE4F529E529C3952A4003021D8C
:101A9D000FE52975F004A42468F9746135F0FA7B1B
:101AAD000190604EEBF0A3EAF0A3E9F0122A6EFF6D
:101ABD00AEF0EE30E71790604EE0FBA3E0FAA3E046
:101ACD00F9EE44408FF0122AD1D21AC21090601A4A
:101ADD00E02529F52980B09078C6E06003021D0F3E
:101AED00906E3CE06003021D0F906E44E0F4FF9099
:101AFD006E3FE0FE6F6003021D0F906E45E0F4FF38
:101B0D00906E40E0FD6F6003021D0F906E46E0F495
:101B1D00FF906E41E06F6003021D0FE4F5298E2BDF
:101B2D00ED6009752908906E40E0F52BE4F52AE586
:101B3D002B20E70F0529E52B25E0F52B052AE52AB6
:101B4D00B408EC906473E0FF131313541FFFE529E1
:101B5D008FF0849064F7F0E5298FF08485F029E506
:101B6D002933333354F8F529906E41E0F52BE4F524
:101B7D002AE52B20E70F0529E52B25E0F52B052A76
:101B8D00E52AB408ECE52925E09078C2F0906E3E88
:101B9D00E020E0079078C2E04401F0907E55744259
:101BAD00F0A37418F09064F7E0907E57F09078C22F
:101BBD00E0907E58F0A37401F0E4A3F07F0612507C
:101BCD008F9078C6740AF0021D0F300702D2019073
:101BDD00601CE0FFA3E09065F8CFF0A3EFF0C20A20
:101BED00021D0F906E40E024C0606C24FE70030255
:101BFD001C7C24F36003021D0F906E3FE070030206
:101C0D001D0F906E42E0FE906E41E07C002400F5C9
:101C1D002DEC3EF52C906014E0652C7004A3E0656E
:101C2D002D6003021D0F302F0D7E097F3E7C607DE0
:101C3D00147B021248E0906015E004F0700690608D
:101C4D0014E004F0125ACF906FBD7403F0E4906568
:101C5D00FAF0A3F0021D0F906E3FE0648060030266
:101C6D001D0FD20E906E3EE0540FF57B021D0F90AE
:101C7D006E3FE06003021D0F906E41E0906F79F0B2
:101C8D00906E42E0906F78F0906E43E0906F77F039
:101C9D00906E44E0906F76F0906E45E0FFC37464F3
:101CAD009FF56CE49078C3F0A3F0D20E906E3EE0F9
:101CBD00540FF57B907E557401F0A37408F0A37456
:101CCD0080F0A37401F0A37406F0906E4163A2013D
:101CDD00907E5A63A2017F04123CD1906E45E0754F
:101CED00F00AA485F02CF52D907E5EF0E52CA3F086
:101CFD007F0B12508F800B906E3DE07002D204C2AC
:101D0D002022301C64E56665616048E56624085450
:101D1D0038FFE56154386F60047E0180027E00E576
:101D2D007D60047D0180027D00EE5D7003021EA9C1
:101D3D000571E571AC707002057014F5828C83E04D
:101D4D00FEE566131313541F2458F8A6068F661567
:101D5D007D80B8C21CC203D2B1200A03021EA99015
:101D6D0065F8E4F0A37414F022300903021EA9A251
:101D7D000182035051E56665616003021EA930B111
:101D8D000AC2B1906019E0906468F030190C30B05F
:101D9D0009906468E06003021EA90571E571AE70DB
:101DAD007002057014F5828E83E0FFE56613131340
:101DBD00541F2458F8A607E56624085438F566150F
:101DCD007DD21CC20122200103021EA990601BE0DE
:101DDD00FE906F7BE0FF6E605C9065FAE07002A391
:101DED00E07054300303021EA9300A04906FBDF059
:101DFD001243F9EF640170367F32125EF6302F0D0B
:101E0D007E0A7F687C6F7D7B7B011248E09065FACE
:101E1D00E4F0A37419F0906FBDE0600214F0906FC0
:101E2D00BDE07078125ACF906FBD7403F022906FA1
:101E3D007BE004F022C217300204125A8922300EC0
:101E4D0007201704125C74229078C3E07002A3E09F
:101E5D00700412526B223018087F081259F5C218FF
:101E6D002220170830160512469C40303010087F8E
:101E7D00091259F5C21022201708301505125B9969
:101E8D00401A301A0512373F4012E566B5610D3024
:0C1E9D000704125E6522200503125D4C54
:011EA9002216
:1039E8009078D8E06022A3E0FEA3E0FFC3E49FFF45
:1039F800E49EFEAB07FA3395E0F9F87F007EC27DBE
:103A0800017C00125B1380219078D9E0FEA3E0FFCF
:103A1800C3E49FFFE49EFEAB07FA3395E0F9F8E4B0
:103A28007F207E1CFDFC125B138F318E308D2F8C16
:103A38002E7BFF7A0A798412316D7BFF7A0A79A688
:103A4800853138853037852F36852E3512316D7B97
:103A5800FF7A0A79E4A211E433F53512316D7BFF60
:103A68007A0B7903A20CE433F53512316D7BFF7ABA
:103A78000B7924A219E433F53512316D7BFF7A0BEB
:103A8800794E906019E075F00AA4FFAEF0E48F3823
:103A98008E37F536F53512316D7535FF75360B7580
:103AA80037777B017A7F796B123167200B14753574
:103AB800FF75360B7537BD7B017A7F796B12594AD2
:103AC80080127535FF75360B7537CC7B017A7F7997
:103AD8006B12594A7B017A7F796B12316D7BFF7AC1
:103AE8000B79DAA20BE433F53512316D7BFF7A0BD3
:103AF80079FB9078C5E0F53512316D7535FF75366F
:103B08001075376F7BFF7A0C791012316D7535FFA0
:103B180075360C75372C753801753905753A0B757E
:103B28003B0D7B017A617952123167753501753623
:103B3800617537527BFF7A0C794512316D7BFF7ABC
:103B48000C7966A207E433F53512316D7BFF7A0CE8
:103B58007986A20DE433F53512316D7BFF7A0C7945
:103B6800A0A20FE433F53512316D90601CE0FEA37E
:103B7800E0FF7C007D061229CD8F357BFF7A0C791A
:103B8800BB12316D7BFF7A0C79F3906473E0FFE42C
:103B98008F38F537F536F53512316D7BFF7A0D79AB
:103BA8003BA214E433F53512316D300B2E7BFF7ACE
:103BB8000D7969A21BE433F53512316D7BFF7A0D5F
:103BC8007996A200E433F53512316D7BFF7A0D79D1
:103BD800C1906F7AE0F53512316D22753501753671
:0D3BE800647537777BFF7A0D79DE12316D41
:013BF50022AD
:103467007E097F3B125494EF4E70037F01227E0D3D
:103477007FF9125494EF4E700302350E12583790AD
:103487007F6E122C59E4FFFEFDFC907F6EE0F8A3DF
:10349700E0F9A3E0FAA3E0FBC3122C486025907F74
:1034A7006EE0F8A3E0A3E0A3E0E47F207E1CFDFC30
:1034B700122BA8122C3A9078D9EEF0A3EFF0E490F3
:1034C70078D8F0E47FB07E04FDFC907F6EE0F8A32F
:1034D700E0F9A3E0FAA3E0FBD3122C484038907838
:1034E700D87401F0907F6EE0F8A3E0A3E0A3E07F3B
:1034F700007EC27D017C00122BA8122C3A9078D94D
:10350700EEF0A3EFF0800F9078D974FFF0A374B8B2
:10351700F0E49078D8F07E0D7FFF125494EF4E6060
:103527000C125E33EF24D024FF92118002C2117E69
:103537000E7F05125494EF4E600C125E33EF24D0C9
:1035470024FF920C8002C20C7E0E7F0B125494EF64
:103557004E600C125E33EF24D024FF92198002C212
:10356700197E0E7F11125494EF4E6013125837E4F0
:103577007B0AFAF9F8122BA8906019EFF08005E49E
:10358700906019F07E0E7F17125494EF4E600C1264
:103597005E33EF24D024FF920B8002D20B7E0E7F86
:1035A7001D125494EF4E600A1258379078C5EFF009
:1035B7008005E49078C5F07E0E7F23125494EF4E79
:1035C700600C125E33EF24D024FF92078002C207FB
:1035D7007E0E7F29125494EF4E600C125E33EF2457
:1035E700D024FF920D8002C20D7E0E7F2F125494BD
:1035F700EF4E600C125E33EF24D024FF920F80024F
:10360700C20F7E0E7F35125494EF4E601612583754
:10361700E47B06FAF9F8122B1D90601CEEF0A3EF7D
:10362700F0800A90601C7402F0A374EEF07E0E7FA7
:103637003B125494EF4E600A125837906473EFF0C0
:1036470080069064737410F07E0E7F41125494EFDD
:103657004E600C125E33EF24D024FF92008002C22A
:10366700007E0E7F47125494EF4E600C125E33EFCC
:1036770024D0906F7AF08005E4906F7AF07E0E7F09
:103687004D125494EF4E600C125E33EF24D024FF9A
:1036970092148002C2147E0E7F53125494EF4E6030
:1036A7000C125E33EF24D024FF921B8002C21B7ED4
:1036B7000E7F59125494EF4E6058E4907F6CF012CD
:1036C7005E33907F6DEFF0643C6047907F6DE0FF65
:1036D700907F6CE0FE04F074772EF582E43464F595
:1036E70083EFF0125E33907F6DEFF0643C600990DA
:1036F7007F6CE0C3948040D3907F6CE0B480021469
:10370700F0907F6CE02477F582E43464F583E4F08D
:103717008023907F6CE0FF04F074772FF582E43408
:1037270064F5837420F0907F6CE02477F582E434AD
:0737370064F583E4F07F005C
:01373E002268
:015F1400226A
:105E7B00BF360BD212E4F54CF54DF568F569BF371B
:045E8B0002C212221B
:1057D900C2A94389029078DAE0FFF58C8F8A75D9DE
:1057E9000475DA4875DB3175DC4975DD4975DE31DB
:1057F900E4F5E9F5F9F5EBF5FB9078D8E060167575
:10580900EC1075ED10E4F5FCF5FD75640875621092
:10581900756301801375EC8075ED80E4F5FCF5FD89
:0E582900756480F562756310E4F5EEF5FE22FD
:0E5EC000E4FFD28C75D84075B740D2AED2AF99
:015ECE0022B1
:0300330002410A7D
:0B410A00C0E0C083C082C0D075D008A8
:10411500C2AF30DC56C3E5EC95EEC395645012E5AD
:104125006325ECF5EC30D70405FC801685FCFC8096
:1041350011C3E5EC9563F5EC30D70415FC800385D8
:10414500FCFC301224854D82854C83E590F0054DAD
:10415500E54D7002054CF582854C83E5EEF0054D85
:10416500E54D7002054C534C0FC2DC30D929301295
:1041750024854D82854C83E590F0054DE54D700213
:10418500054CF582854C83E5EBF0054DE54D700258
:10419500054C534C0FC2D930DA6AE562700405FC50
:1041A5008010E56225ECF5EC30D70405FC8003852D
:1041B500FCFC30134DE54E5480F54BE54E25E0F5FE
:1041C5004E309702054E201103634E01303A19E532
:1041D5004E656A6006E54E65677027756000756512
:1041E50000854E50C23A801A0565E5655407701280
:1041F50053653FE565131313541F2450F8A64E75F8
:104205004E00C2DA30DB71E562700405FD8010E511
:104215006225EDF5ED30D70405FD800385FDFDE54F
:104225006665616029E56154077013E56113131331
:10423500541F2458F8E6F54F200C03634FFFE54F54
:10424500339296E54F25E0F54F056153613FB292F4
:10425500301223854D82854C83E590F0054DE54D63
:104265007002054CF582854C83E4F0054DE54D70F3
:0A42750002054C534C0FC2DBD2AF20
:09427F00D0D0D082D083D0E0320F
:10530600021EAAE493A3F8E493A34003F68001F2F5
:1053160008DFF48029E493A3F85407240CC8C333A8
:10532600C4540F4420C8834004F456800146F6DF77
:10533600E4800B0102040810204080905CFAE47EB1
:10534600019360BCA3FF543F30E509541FFEE4936C
:10535600A360010ECF54C025E060A840B8E493A333
:10536600FAE493A3F8E493A3C8C582C8CAC583CA5E
:10537600F0A3C8C582C8CAC583CADFE9DEE780BE16
:015D22000080
:10295300BB010689828A83E0225002E722BBFE0282
:09296300E32289828A83E49322B5
:10296C00BB010CE58229F582E5833AF583E0225020
:10297C0006E92582F8E622BBFE06E92582F8E2226A
:0D298C00E58229F582E5833AF583E4932284
:10299900BB010689828A83F0225002F722BBFE011D
:0229A900F32217
:1029AB00F8BB010DE58229F582E5833AF583E8F062
:1029BB00225006E92582C8F622BBFE05E92582C80E
:0229CB00F222F6
:1029CD00BC000BBE0029EF8DF084FFADF022E4CCEE
:1029DD00F875F008EF2FFFEE33FEEC33FCEE9DECB7
:1029ED00984005FCEE9DFE0FD5F0E9E4CEFD22EDFD
:1029FD00F8F5F0EE8420D21CFEADF075F008EF2F47
:102A0D00FFED33FD4007985006D5F0F222C398FD37
:052A1D000FD5F0EA22D4
:102A2200C2D5EC30E709B2D5E4C39DFDE49CFCEECF
:102A320030E715B2D5E4C39FFFE49EFE1229CDC351
:102A4200E49DFDE49CFC80031229CD30D507C3E44C
:062A52009FFFE49EFE223E
:102A5800C5F0F8A3E028F0C5F0F8E5821582700209
:062A68001583E038F022A6
:102A6E00BB010A89828A83E0F5F0A3E02250068733
:102A7E00F009E71922BBFE07E3F5F009E3192289F5
:0B2A8E00828A83E493F5F07401932228
:102A9900BB0110E58229F582E5833AF583E0F5F07B
:102AA900A3E0225009E92582F886F008E622BBFE58
:102AB9000AE92582F8E2F5F008E222E5832AF5839E
:082AC900E993F5F0A3E9932263
:102AD100BB010A89828A83F0E5F0A3F0225006F750
:0F2AE10009A7F01922BBFE06F3E5F009F319224D
:102AF000F8BB0111E58229F582E5833AF583E8F018
:102B0000E5F0A3F0225009E92582C8F608A6F022D4
:0D2B1000BBFE09E92582C8F2E5F008F222BB
:102B1D00E88FF0A4CC8BF0A42CFCE98EF0A42CFC57
:102B2D008AF0EDA42CFCEA8EF0A4CDA8F08BF0A4D5
:102B3D002DCC3825F0FDE98FF0A42CCD35F0FCEB34
:102B4D008EF0A4FEA9F0EB8FF0A4CFC5F02ECD39F9
:0F2B5D00FEE43CFCEAA42DCE35F0FDE43CFC2266
:102B6C0075F008758200EF2FFFEE33FECD33CDCC20
:102B7C0033CCC58233C5829BED9AEC99E5829840A3
:102B8C000CF582EE9BFEED9AFDEC99FC0FD5F0D680
:102B9C00E4CEFBE4CDFAE4CCF9A88222B800C1B9AA
:102BAC000059BA002DEC8BF084CFCECDFCE5F0CBE8
:102BBC00F97818EF2FFFEE33FEED33FDEC33FCEB21
:102BCC0033FB10D703994004EB99FB0FD8E5E4F9DC
:102BDC00FA227818EF2FFFEE33FEED33FDEC33FCC9
:102BEC00C933C910D7059BE99A4007EC9BFCE99ABD
:102BFC00F90FD8E0E4C9FAE4CCFB2275F010EF2F02
:102C0C00FFEE33FEED33FDCC33CCC833C810D70701
:102C1C009BEC9AE899400AED9BFDEC9AFCE899F83C
:0E2C2C000FD5F0DAE4CDFBE4CCFAE4C8F922CF
:105B1300C2D5E830E70FB2D5E4C39BFBE49AFAE4BD
:105B230099F9E498F8EC30E717B2D5125B49122BD8
:105B3300A8E4C39BFBE49AFAE499F9E498F8800398
:105B4300122BA830D50DE4C39FFFE49EFEE49DFD18
:045B5300E49CFC22B0
:0E2C3A00C3E49FFFE49EFEE49DFDE49CFC22AB
:102C4800EB9FF5F0EA9E42F0E99D42F0E89C45F0E2
:012C58002259
:0C2C5900ECF0A3EDF0A3EEF0A3EFF022EE
:102C6500A8828583F0D083D082122C7C122C7C1212
:102C75002C7C122C7CE473E493A3C583C5F0C58337
:102C8500C8C582C8F0A3C583C5F0C583C8C582C8B9
:012C9500221C
:10310B00E5412435F8E6054122783230380278352E
:10311B00E475F001122C960229532031EB7F2ED24D
:10312B00318018EF540F2490D43440D4FF30350B3A
:10313B00EF24BFB41A0050032461FFE5426002156F
:10314B00420545E5457002054430380D7832E4758B
:10315B00F001122C96EF022999025A407403D238CF
:10316B008003E4C238F5418B328A338934E4F5426B
:10317B00F544F545E54260077F2012314680F57531
:10318B0043FFC232C231C233C234C236C237C23934
:10319B00123114FF700D3038057F00123157AF45D7
:1031AB00AE4422B4255FC2D5C235123114FF24D0F0
:1031BB00B40A00501A75F00A784230D50508B6FFEC
:1031CB000106C6A426F620D5047002D23480D92479
:1031DB00CFB41A00EF5004C2E5D235023357D232C6
:1031EB0080C6D23180C0D23380BCD2D580BAD23621
:1031FB0080B47F201231462033077401B542004062
:10320B00F112310BFF12314602317FD239D23780A6
:10321B009512310BFB12310BFA12310BF94A4B7031
:10322B000679287A347BFF20332EE542602A7E0014
:10323B008E8275830012296C60060EEE654370F06A
:10324B00C2D5EBC0E0EAC0E0E9C0E0EE12339ED09D
:10325B00E0F9D0E0FAD0E0FB122953FF60AAEBC0F3
:10326B00E0EAC0E0E9C0E0123146D0E02401F9D039
:10327B00E03400FAD0E0FBE5430460DCD543D980B1
:10328B00877BFF7A33799AD233809C7910800279CD
:10329B0008C237C2398008D2D5790A8004790AC2AC
:1032AB00D5E543047002F543E4FAFDFEFF12310B42
:1032BB00FC7B0820321312310BFD7B1030310A12CC
:1032CB00310BFE12310BFF7B20EC3382D592D550A4
:1032DB0013C3E43031069FFFE49EFEE42032039DCE
:1032EB00FDE49CFCE4CBF8C232EC700CCFCECDCC21
:1032FB00E824F8F870F38017C3EF33FFEE33FEEDDD
:10330B0033FDEC33FCEB33FB994002FB0FD8E9EBBD
:10331B00303205F8D0E0C448B232C0E00AEC4D4E72
:10332B004F78207B0070C2EAB5430040BCC0E0126E
:10333B0033A0D0F0D0E0203204C4C0E0C4B232C01D
:10334B00F012312FD0F0D5F0EB02317F122CF53289
:10335B001C5332965831ED4C31E942329A4F32A21E
:0F336B004432A24932024332A855328C46328C8A
:10337A0045328C4734485031F12D31F52E32182B15
:10338A0031F92332162034312A31B1480000321083
:10339A003F3F3F00790AA2D5203414303609B910CC
:1033AA00020404B9080104A2D520370250010420FE
:1033BA0033689233B542005034C0E07F203034196C
:1033CA007F30A23372377236500F1233F7C233C2CC
:1033DA0037C236C2397F30800F303603E9C0E01277
:1033EA003146303603D0E0F9D0E0B542CC3036175A
:1033FA007F30B9100C1231467F583035077F7880FC
:10340A0003B908031231463033057F2D0231467F56
:10341A00202039F87F2B2037F322923380CF286E71
:10342A00756C6C2900D23212310B3032F8C2327804
:10343A004230D50108F60231B12D504349581231B4
:10344A000B2403B405004001E4903443931231374E
:0D345A00743A123137D234754204023296B2
:105E8F00C3EE6480948040028007C3E49FFFE49ECA
:025E9F00FE22E1
:10594A008B328A3389348B388A39893AAB320534B7
:10595A00E534AA337002053314F912295370ED7431
:10596A00FF2534F53474FF3533F533AB350537E5A8
:10597A0037AA367002053614F9122953FFAB3205DD
:10598A0034E534AA337002053314F9EF12299970F9
:08599A00DAAB38AA39A93A2260
:103DDF008B2E8A2F8930E4F53AF539F538F537F51A
:103DEF0035F536E532453345316012EBC0E0EAC0B8
:103DFF00E0E9C0E0AB31AA32A933122CA6AB2E05F5
:103E0F0030E530AA2F7002052F14F9122953F53B14
:103E1F00C394094007E53BD3940D40E1E53B642093
:103E2F0060DBE53BB42D054336038016E53BB42B31
:103E3F0005433601800C74FF2530F53074FF352FA4
:103E4F00F52FE53460046410703FAB2EAA2FA93014
:103E5F0012295364306009E534702E75340A8029B5
:103E6F0090000112296CFF64786004EFB45813437B
:103E7F00360175341074022530F530E4352FF52FE7
:103E8F008007E5347003753408AB2E0530E530AA92
:103E9F002F7002052F14F9122953F53BC39461407B
:103EAF000AE53BD3947A5003533BDF74D0253BF59F
:103EBF003BC3940A400CE53B9411406D74F9253BCC
:103ECF00F53BE53BD395345060433601853A3F854A
:103EDF00393E85383D85373CAF347E00E4FCFDAB81
:103EEF003AAA39A938A837122B1DC8ECC8C9EDC991
:103EFF00CAEECACBEFCBE4FCFDFEEB253BF53AEE69
:103F0F003AF539ED39F538EC38F537AF3AAE39AD1A
:103F1F0038FCAB3FAA3EA93DA83CD3122C48500316
:103F2F00023E98433604023E98E53620E003E480D3
:103F3F002DE53245334531601EAB2EE53024FFF9B8
:103F4F00E52F34FFFAEBC0E0EAC0E0E9C0E0AB31A7
:103F5F00AA32A933122CA6E53630E20774FFFFFE12
:103F6F00FDFC22E536AF3AAE39AD38AC3730E10360
:043F7F00022C3A22B4
:102C9600FAE6FB0808E6F925F0F618E6CA3AF6223F
:102CA600BB011A89828A83D0F0D0E0F8D0E0F9D04F
:102CB600E0FAD0E0FBE8C0E0C0F0022D245016E9AF
:102CC600F8D083D082D0E0F9D0E0FAD0E0FBC08221
:102CD600C083022D1BBBFE16E9F8D083D082D0E05C
:0F2CE600F9D0E0FAD0E0FBC082C083022D2D228E
:102CF500D083D082F8E4937012740193700DA3A36E
:102D050093F8740193F5828883E473740293686081
:062D1500EFA3A3A380DF81
:092D1B00EBF608EAF608E9F622DD
:092D2400EBF0A3EAF0A3E9F022B0
:092D2D00EBF208EAF208E9F222D7
:00000001FF
